:100000000C9471090C94A9090C94A9090C94A909E0
:100010000C94A9090C94A9090C94A9090C94A90998
:100020000C94A9090C94A9090C94DB2B0C94972B24
:100030000C942E2D0C94A9090C94A9090C94A909CF
:100040000C94A9090C94A9090C94A9090C94A90968
:100050000C94A9090C940A2D0C94A9090C94A909D3
:100060000C94A9090C94A9090C94A9090C94A90948
:100070000C94A9090C94A9090C94A9090C94A90938
:100080000C94A9090C94A9090C94A9090C94A90928
:100090000C94A9090C94A9090C94A9090C94A90918
:1000A0000C94A9090C94A9090C94A9090631FF091B
:1000B00074A1010975150026FF00952075088102BD
:1000C0000976150026FF00952075089102C00501EC
:1000D0000902A10185020901A100050919012908E8
:1000E00015002501950875018102050109300931C6
:1000F0001581257F95027508810609381581257FB0
:10010000950175088106050C0A38021581257F9531
:100110000175088106C0C005010980A10185031988
:10012000012AB700150126B700950175108100C09E
:10013000050C0901A101850419012AA00215012657
:10014000A002950175108100C00660FF0961A10140
:100150000962150026FF00952075088102096315C4
:100160000026FF00952075089102C005010906A12F
:1001700001050719E029E71500250195087501819A
:10018000029501750881010507190029FF15002650
:10019000FF009506750881000508190129059505D8
:1001A00075019102950175039101C00000000000E6
:1001B000000000000000000000000000000000003F
:1001C0000000000000000000000000000000007EB1
:1001D0000F00D4FFFFFFC700000078000000000000
:1001E0000000002A2B280000000000000000000092
:1001F00000000000000029000000002C1E34202117
:100200002224342627252E362D3738271E1F20215D
:1002100022232425263333362E37381F04050607BC
:1002200008090A0B0C0D0E0F1011121314151617D6
:1002300018191A1B1C1D2F3130232D3504050607F4
:1002400008090A0B0C0D0E0F1011121314151617B6
:1002500018191A1B1C1D2F3130354C7267626C69DE
:100260006768742064697361626C65205B45455002
:10027000524F4D5D3A207267626C696768745F63C4
:100280006F6E6669672E656E61626C65203D202524
:10029000750A007267626C6967687420656E6162D6
:1002A0006C65205B454550524F4D5D3A2072676248
:1002B0006C696768745F636F6E6669672E656E61EF
:1002C000626C65203D2025750A007267626C696763
:1002D000687420746F67676C65205B454550524FAA
:1002E0004D5D3A207267626C696768745F636F6E18
:1002F0006669672E656E61626C65203D2025750A12
:100300000044454255473A2064697361626C6564F4
:100310002E0A0044454255473A20656E61626C657D
:10032000642E0A003F00433E20004F6E6573686FE5
:10033000743A206163746976653A2025640A000A7C
:10034000002530325820006B6579626F6172645FFE
:100350007265706F72743A20007267626C696768C8
:10036000745F636F6E6669672E7370656564203DA8
:100370002025640A007267626C696768745F636F46
:100380006E6669672E76616C203D2025640A0072D6
:1003900067626C696768745F636F6E6669672E7306
:1003A0006174203D2025640A007267626C69676889
:1003B000745F636F6E6669672E687565203D2025E2
:1003C000640A007267686C696768745F636F6E6661
:1003D00069672E6D6F6465203D2025640A00726791
:1003E000626C696768745F636F6E6669672E656EBD
:1003F00061626C65203D2025640A007267626C6949
:100400006768745F636F6E66696720454550524F39
:100410004D3A0A007267626C696768745F696E6959
:1004200074207267626C696768745F636F6E666977
:10043000672E6D6F6465203D20302E2057726974E1
:10044000652064656661756C742076616C75657392
:1004500020746F20454550524F4D2E0A007267623E
:100460006C696768745F696E6974206565636F6E37
:10047000666967206973206E6F7420656E61626CB7
:1004800065642E0A007267626C696768745F696EE2
:100490006974207374617274210A007267626C69F6
:1004A0006768745F696E69742063616C6C65642E43
:1004B0000A005B735D000A00253033326C62003A3B
:1004C000200025303258000A722F63203031323339
:1004D000343536373839414243444546303132337A
:1004E0003435363738394142434445460A001E0FF9
:1004F0000500047F3F1F643214643214783C1E1ED2
:10050000140A050A0025303258006C65645F746176
:10051000736B3A20007267626C6967687420646963
:100520007361626C65205B4E4F454550524F4D5D87
:100530003A207267626C696768745F636F6E6669A0
:10054000672E656E61626C65203D2025750A00721C
:1005500067626C6967687420656E61626C65205BB8
:100560004E4F454550524F4D5D3A207267626C695F
:100570006768745F636F6E6669672E656E61626C33
:1005800065203D2025750A007267626C6967687492
:1005900020736574207370656564205B4E4F45451C
:1005A00050524F4D5D3A2025750A00290A002575E5
:1005B000002F002575005D280025640020002564BB
:1005C00000200025640020002564007C00253032D6
:1005D00058006D6F7573656B6579205B62746E7C16
:1005E000782079207620685D287265702F61636CB1
:1005F000293A205B00000101010101010101010212
:1006000002020202020202020303030303030303C2
:10061000040404040404040505050505060606068D
:1006200006070707070708080808090909090A0A49
:100630000A0B0B0B0C0C0C0D0D0D0E0E0E0F0F0FED
:100640001010111111121213131414151516161778
:1006500017181819191A1A1B1B1C1D1D1E1E1F20E6
:1006600020212222232424252626272829292A2B33
:100670002C2D2D2E2F303132323334353637383958
:100680003A3B3C3D3E3F4041424344454647484952
:100690004A4C4D4E4F50515354555658595A5B5D24
:1006A0005E5F616264656668696B6C6D6F707273C2
:1006B0007577787A7B7D7E8082838587888A8C8E29
:1006C0008F91939596989A9C9EA0A2A3A5A7A9AB5B
:1006D000ADAFB1B3B5B7BABCBEC0C2C4C6C9CBCD4D
:1006E000CFD1D4D6D8DBDDDFE2E4E7E9EBEEF0F3FF
:1006F000F5F8FAFDFF7267626C69676874207469C7
:100700006D657220656E61626C65642E0A007267A9
:10071000626C69676874206D6F6465205B4E4F453D
:100720004550524F4D5D3A2025750A007267626C44
:1007300069676874206D6F6465205B454550524F52
:100740004D5D3A2025750A007267626C69676874AE
:100750002073657420687376205B4E4F4545505278
:100760004F4D5D3A2025752C25752C25750A007294
:1007700067626C696768742073657420687376209B
:100780005B454550524F4D5D3A2025752C25752C03
:1007900025750A007267626C696768742072616906
:1007A0006E626F7720736574206873763A202564D3
:1007B0002C25642C25642C25750A00FFAA7F554042
:1007C0007267626C696768742074696D6572206411
:1007D000697361626C652E0A002223252628292A66
:1007E0002C2D2F3032333536383A3B3D3E40424394
:1007F0004547494A4C4E5051535557595A5C5E60D3
:1008000062646668696B6D6F71737577797B7D7FE4
:1008100081838587898A8C8E90929496989A9C9EE3
:100820009FA1A3A5A7A8AAACAEAFB1B3B4B6B8B9FF
:10083000BBBCBEBFC1C2C3C5C6C7C9CACBCCCDCE67
:10084000D0D1D2D2D3D4D5D6D7D7D8D9D9DADADB4A
:10085000DBDBDCDCDCDCDCDDDDDDDDDCDCDCDCDCD6
:10086000DBDBDBDADAD9D9D8D7D7D6D5D4D3D2D215
:10087000D1D0CECDCCCBCAC9C7C6C5C3C2C1BFBEFD
:10088000BCBBB9B8B6B4B3B1AFAEACAAA8A7A5A368
:10089000A19F9E9C9A98969492908E8C8A89878527
:1008A00083817F7D7B79777573716F6D6B69686606
:1008B0006462605E5C5A5957555351504E4C4A49D8
:1008C00047454342403E3D3B3A3836353332302F80
:1008D0002D2C2A2928262523226B65796D61705FCE
:1008E000636F6E6669672E7261773A2025303258E1
:1008F0000A2E737761705F636F6E74726F6C5F63E3
:100900006170736C6F636B3A2025750A2E6361709A
:10091000736C6F636B5F746F5F636F6E74726F6C19
:100920003A2025750A2E737761705F6C63746C5F73
:100930006C6775693A2025750A2E737761705F724E
:1009400063746C5F726775693A2025750A2E737738
:1009500061705F6C616C745F6C6775693A202575B6
:100960000A2E737761705F72616C745F726775696C
:100970003A2025750A2E6E6F5F6775693A202575D6
:100980000A2E737761705F67726176655F65736366
:100990003A2025750A2E737761705F6261636B730D
:1009A0006C6173685F6261636B73706163653A2049
:1009B00025750A2E6E6B726F3A2025750A006465E4
:1009C0006275675F636F6E6669672E7261773A2042
:1009D000253032580A2E656E61626C653A202575A5
:1009E0000A2E6D61747269783A2025750A2E6B653E
:1009F00079626F6172643A2025750A2E6D6F757386
:100A0000653A2025750A006565636F6E6669673A09
:100A10000A64656661756C745F6C617965723A2011
:100A200025750A000A092D204D61676963202D0A8A
:100A3000443A094465627567204D65737361676563
:100A400020546F67676C650A583A094D6174726982
:100A500078204465627567204D6F646520546F6728
:100A6000676C65202D2053686F77206B65797072F5
:100A7000657373657320696E206D61747269782087
:100A8000677269640A4B3A094B6579626F617264F7
:100A900020446562756720546F67676C65202D2060
:100AA00053686F77206B6579707265737320726518
:100AB000706F72740A4D3A094465627567204D6F14
:100AC00075736520546F67676C650A563A095665F9
:100AD0007273696F6E0A533A095374617475730ABD
:100AE000433A09416374697661746520436F6E739C
:100AF0006F6C65204D6F64650A46312D4631303A82
:100B00000953776974636820746F204C617965724A
:100B100020302D392028463130203D204C30290A04
:100B2000302D393A0953776974636820746F204C0B
:100B30006179657220302D390A47524156453A098C
:100B400053776974636820746F204C6179657220F3
:100B5000302028616C7465726E617465290A423AAE
:100B6000094A756D7020746F20426F6F746C6F61ED
:100B70006465720A4553433A094A756D7020746F73
:100B800020426F6F746C6F616465722028616C74B1
:100B900065726E617465290A453A095072696E740E
:100BA00020454550524F4D2053657474696E6773EC
:100BB0000A4253504143453A09436C6561722045EE
:100BC0004550524F4D0A000A092D20436F6E736F36
:100BD0006C65202D0A4553432F713A09717569746C
:100BE0000A6D3A096D6F7573656B65790A000A09BC
:100BF0002D2056657273696F6E202D0A5649443A4E
:100C00002030783433343428436861727565204469
:100C1000657369676E29205049443A20307835332E
:100C200033352853756E736574746572205232299A
:100C3000205645523A203078303030310A425549FA
:100C40004C443A202028417567202035203230322C
:100C500032290A4F5054494F4E533A204C55464181
:100C6000204D4F5553454B45592045585452414B03
:100C7000455920434F4E534F4C4520434F4D4D4116
:100C80004E44204C544F20343039360A4743433ABF
:100C900020382E352E30204156522D4C4942433AB1
:100CA00020322E302E30204156525F415243483A76
:100CB00020617672350A000A092D2053746174751B
:100CC00073202D0A686F73745F6B6579626F617250
:100CD000645F6C65647328293A20253032580A6BAA
:100CE0006579626F6172645F70726F746F636F6C4D
:100CF0003A20253032580A6B6579626F6172645F01
:100D000069646C653A20253032580A74696D6572E1
:100D10005F72656164333228293A202530386C5877
:100D20000A003F000A6D6F7573653A206F66660AA8
:100D3000000A6D6F7573653A206F6E0A000A6B6565
:100D400079626F6172643A206F66660A000A6B65A9
:100D500079626F6172643A206F6E0A000A6D617485
:100D60007269783A206F66660A000A6D617472696A
:100D7000783A206F6E0A000A64656275673A206FE0
:100D800066660A000A64656275673A206F6E0A003B
:100D90000A0A4A756D70696E6720746F20626F6F02
:100DA000746C6F616465722E2E2E2000433E20000D
:100DB000436C656172696E6720454550524F4D0A1C
:100DC00000313A0964656C6179282A31306D7329E4
:100DD0003A2025750A323A09696E74657276616C3B
:100DE000286D73293A2025750A333A096D61785FB9
:100DF00073706565643A2025750A343A0974696D23
:100E0000655F746F5F6D61783A2025750A353A0920
:100E1000776865656C5F6D61785F73706565643A6E
:100E20002025750A363A09776865656C5F74696DC7
:100E3000655F746F5F6D61783A2025750A00703ABE
:100E4000097072696E742076616C7565730A643A14
:100E5000097365742064656661756C74730A7570D6
:100E60003A092B310A646E3A092D310A6C743A0939
:100E70002B31300A72743A092D31300A4553432F11
:100E8000713A09717569740A0A7370656564203D69
:100E90002064656C7461202A206D61785F737065D1
:100EA0006564202A2028726570656174202F207483
:100EB000696D655F746F5F6D6178290A7768657227
:100EC000652064656C74613A20637572736F723D5E
:100ED00025642C20776865656C3D25640A5365653B
:100EE00020687474703A2F2F656E2E77696B697065
:100EF000656469612E6F72672F77696B692F4D6F1B
:100F00007573655F6B6579730A004D3E20004D2552
:100F1000753A25733E20003F0A003D2025750A00E2
:100F20003F0A0064656661756C74730A0025750A72
:100F3000003F0A000A092D2056616C756573202D4B
:100F40000A00710A000A092D204D6F7573656B65E3
:100F500079202D0A004C25640A003A003B00165CFB
:100F60001E001F0020002100220023002400250075
:100F7000260027002D002E0035002A003C003D00F1
:100F80002B0014001A000800150017001C001800A0
:100F90000C00120013002F0030003100A9003E00A9
:100FA0003F00390004001600070009000A000B008A
:100FB0000D000E000F00330034002800AA000000CE
:100FC00040004100E10031001D001B000600190037
:100FD000050011001000360037003800E500A800B9
:100FE000520042004300E000E300E2000151000033
:100FF0002C00000000002C000000E6005000510012
:101000004F00AB0044004500005C1E001F002000A4
:1010100021002200230024002500260027002D00A7
:101020002E0035002A00680069002B0014001A0009
:101030000800150017001C0018000C001200130017
:101040002F0030003100A9006A006B003900040055
:101050001600070009000A000B000D000E000F002B
:10106000330034002800AA0000006C006D00E1008D
:1010700031001D001B0006001900050011001000C2
:10108000360037003800E500A80052006E006F00FF
:10109000E000E300E200010000002C00000000007E
:1010A0002C000000E600500051004F00AB00010092
:1010B0000100010001000100010001000100010028
:1010C0000100010001000100010001000100010018
:1010D0000100010001000100010001000100010008
:1010E00001000100010001000100010001000100F8
:1010F00001000100010001000100010001000100E8
:1011000001000100010001000100010001000100D7
:1011100001000000010001000100010001000100C8
:1011200001000100010001000100010001000100B7
:1011300001000100010001000100E00001000100C8
:10114000010000000100000000000100000001009B
:101150000100010001000100010001000100010087
:101160000100010001000100010001000100010077
:101170000100010001000100010001000100010067
:101180000100010001000100010001000100010057
:101190000100010001000100010001000100010047
:1011A0000100010001000100010001000100010037
:1011B0000100010001000100010001000000010028
:1011C0000100010001000100010001000100010017
:1011D0000100010001000100010001000100010007
:1011E00001000100E0000100010001000000010019
:1011F00000000000010000000100010001000100EA
:1012000001005B435D005B445D005B535D005B5729
:101210005D005B525D0009027B00040100A0FA0939
:101220000400000103010100092111010001224015
:101230000007058103080001090401000203000002
:10124000000921110100012222000705820320006C
:101250000107050303200001090402000103000047
:1012600000092111010001227B00070584032000F1
:10127000010904030002030000000921110100011B
:101280002222000705850320000107050503200031
:10129000011201000200000008444335530100011F
:1012A0000200011A03530075006E0073006500749C
:1012B0000074006500720020005200320000001C23
:1012C000034300680061007200750065002000445F
:1012D0000065007300690067006E000000040309E8
:1012E000040011241FBECFEFDAE0DEBFCDBF04B68D
:1012F00003FE18C080915C0390915D03A0915E0392
:10130000B0915F038730904BA740B04B59F41092D7
:101310005C0310925D0310925E0310925F03E0E0A5
:10132000F8E3099523E0A8E0B2E001C01D92AC35D6
:10133000B207E1F712E0A0E0B1E0E8E1FCE602C0AC
:1013400005900D92A830B107D9F70E94552D0C9445
:10135000E1350C940000FF93EF93E0910802F091C7
:101360000902309709F00995EF91FF910895FC016A
:101370008591803011F0EFDFFBCF0895FF27E0E289
:1013800030E247FF0CC0419597FF09C0EDE2609540
:10139000709580959095611D711D811D911D27FF90
:1013A00002C0219530E350E2AA27660F771F881FFD
:1013B000991FAA1FA41710F0A41B63955A95A9F7AB
:1013C000AA3008F0A95FA05DAF93F3956115710590
:1013D0008105910541F7ED3211F4EF93F395F21782
:1013E00018F43F93F395FBCF8F91B5DFFA95E1F7B2
:1013F0000895E991F9918591803021F0853219F0B5
:10140000AADFF9CF089520E0E89455915532C1F351
:10141000503311F4689455915A3348F4505390F373
:10142000220F022E220F220F200D250FF4CF0EF4D3
:10143000219589919991533619F3533729F15335F1
:1014400059F1BC0188279927E8945C3621F48991E9
:10145000999168945591543639F446EF7EF077FFB0
:101460000DC08FEF9FEF0AC055374AE039F058356D
:1014700040E121F0523642E009F00895FF93EF93E6
:101480007DDFEF91FF91B7CFFF93EF93FC01819147
:101490008030B9F360DFFBCFFF93EF9368DFF1CFCC
:1014A000DF93CF93CDB7DEB72596A3DFCF91DF9142
:1014B0000895E8EDF0E080818E7F80831092E20055
:1014C0001092DA001092E100A0EEB0E08C91816001
:1014D0008C9380818F77808319BCA7EDB0E08C91CD
:1014E0008E7F8C9380818F7E80831092410308953C
:1014F0002091E4003091E50095E6A9012091EC00EF
:10150000822F817020FF06C08091E80080FF06C016
:1015100080E008952091E80022FD1AC080914E03DA
:10152000882389F0853089F08091EB0085FD0FC01C
:101530002091E4003091E50042175307F9F29150F1
:10154000E1F684E0089582E0089583E0089581E063
:101550000895EF92FF920F931F93CF937C018B011D
:101560000E94780AC82F811117C08091E80085FD7C
:101570000BC08091E8008E778093E8000E94780A83
:10158000882399F3C82F08C0F70181917F018093C8
:10159000F1000150110949F78C2FCF911F910F9144
:1015A000FF90EF9008958091500387FF13C08091C2
:1015B000E80082FF06C08091E8008B778093E80006
:1015C00004C080914E038111F2CF089580914E03A3
:1015D0008823D9F38091E80080FFF8CF8091E8005C
:1015E0008E77ECCF982F9093E900242F762F50E040
:1015F000891731F07091EC002091ED005091F000CE
:1016000021FD07C09F5F973071F78093E90081E06B
:1016100008953091EB003E7F3093EB003091ED0068
:101620003D7F3093ED003091EB0031603093EB0063
:101630007093EC002093ED005093F0002091EE00A9
:1016400027FDE0CF80E00895B0E0A0E0EAE2FBE013
:101650000C949334C8EDD0E088818F7E8883E7EDC9
:10166000F0E080818160808384E082BF81E08093AC
:10167000410388818E7F888302EE10E0F80110829A
:101680001092DA0081EEC82ED12CF60110828881EA
:101690008F77888388818068888388818F7D88831D
:1016A00019BC10924E0310924F0310924D031092EA
:1016B0004C0390EEE92EF12CF70180818B7F808323
:1016C00088818160888342E060E080E00E94F20AC5
:1016D000F60180818E7F8083F80180818160808324
:1016E000808188608083F70180818E7F80838881FC
:1016F00080618883CDB7DEB7E8E00C94AF34FC019D
:10170000809156039091570386179707A0F06115B3
:10171000710529F49091E8009E779093E80090E09D
:101720006115710551F4911108C08091E80082FFA4
:1017300034C080E00895BC01F2CF80914E0388232D
:10174000C1F18530C1F18091E80083FD30C0809106
:10175000E80082FDEACF8091E80080FFE1CF809130
:10176000F3002091F200382F6115710519F028302F
:10177000310558F091E02830310509F090E02091D2
:10178000E8002E772093E800CBCF81918093F10081
:10179000615071092F5F3F4FE7CF80914E0388233F
:1017A00041F0853041F08091E80083FFBECF81E0B9
:1017B000089582E0089583E0089508958091430399
:1017C00008959C014FB7F8948091370390913803A6
:1017D000A0913903B0913A034FBF821B930B089538
:1017E0002FB7F8948091370390913803A091390373
:1017F000B0913A032FBF08952091340330913503FF
:101800002817390771F09093350380933403E091E2
:101810003203F0913303309721F00084F185E02DFD
:101820000995089520913003309131032817390725
:1018300071F09093310380933003E0913203F09183
:101840003303309721F00680F781E02D0995089544
:10185000E0913203F0913303309729F00190F08149
:10186000E02D0995089580E00895FA01811101C0E5
:10187000FB0109950895089580912403982F9E7F78
:1018800029F4817082608093240308958635E8F3FB
:1018900081708465F8CFAF92BF92DF92EF92FF9292
:1018A0000F931F93CF93DF93082F162FE901E42F97
:1018B000F0E0EB50FA4F611110C0E4915E2F4E2F13
:1018C0004983E8835A83DF91CF911F910F91FF9055
:1018D000EF90DF90BF90AF900895E62EF12C4491E9
:1018E000D42EE42FF0E026E0829FC00111242FEFD8
:1018F00030E0B9010E944534802F90E0880F991F95
:1019000055E5569FD001579FB00D11248A1B9B0BA4
:10191000982F990F890F5901AE18BF08AE9ED001BC
:10192000AF9EB00DBE9EB00D11245B2F189F80019D
:101930001124012F11275901A01AB10AAE9E80016E
:10194000AF9E100DBE9E100D11245901A81AB108AA
:10195000AE9CC001AF9C900DBE9C900D1124892FB0
:101960009927281B390B2E9FC0012F9F900D3E9F5A
:10197000900D1124E92F62307105A1F050F461152A
:10198000710509F49DCF6130710581F0EB2F512F66
:1019900097CF6430710569F080F06630710509F405
:1019A0008FCFF4CFE42F4B2F592F8ACFE42F412F25
:1019B00087CFEB2F542F492F83CF4B2F5D2DE12F56
:1019C0007FCF4091C502803F59F48091C60287FFC6
:1019D0000DC01092C60241110BC01092BE0208C089
:1019E000813F81F48091C60218169CF3442381F054
:1019F0008091C7029091C802892B09F05AC01092B9
:101A0000BC020895823F49F447FFF0CF1092C5020F
:101A10008091C6028111ECCFE0CF833F19F41416F8
:101A2000ACF3E4CF9091C702893F29F41916F4F67C
:101A30001092C702DBCF8A3F19F497FFD7CFF8CFB8
:101A40009091C8028B3F29F497FFD0CF1092C80223
:101A5000CDCF8C3F19F41916CCF3C8CF9CE0980F6A
:101A6000953090F4845F990B21E030E0B90102C019
:101A7000660F771F8A95E2F7CB0180959091C4029B
:101A800089238093C402B2CF8D3F31F48091BD028F
:101A90008E7F8093BD02AACF8E3F21F48091BD023C
:101AA0008D7FF7CF8F3F09F0A1CF8091BD028B7F53
:101AB000F0CF08958091BD0280FF0CC060911F019E
:101AC00070E075956795759567956115710549F194
:101AD000862F089581FF06C060911F0170E0759503
:101AE0006795F3CF60911F0182FD0BC09091BC02FE
:101AF0009923A1F060911E0180911F01961738F083
:101B0000682F70E06038710500F38FE70895899FB2
:101B1000C001112470E00E945934F4CF61E070E0FC
:101B2000D7CF81E008958091BD0280FF0DC0609104
:101B3000210170E0660F771F6038710570F561153F
:101B4000710569F1862F089581FF07C06091210119
:101B500084E0689FB0011124EFCF82FF04C0609140
:101B6000210188E0F6CF8091BE02882399F0209170
:101B70002001609121018217A0F7869FC0011124E6
:101B800033E0880F991F3A95E1F7622F70E00E94C9
:101B90005934D2CF68E070E0D5CF8FE7089581E067
:101BA0000895803F31F40E94930D81958093C60281
:101BB0000895813F19F40E94930DF8CF823F31F4CC
:101BC0000E94930D81958093C5020895833F19F477
:101BD0000E94930DF8CF893F29F40E945A0D8093FB
:101BE000C70208958A3F21F40E945A0D8195F7CFCC
:101BF0008B3F31F40E945A0D81958093C80208955D
:101C00008C3F19F40E945A0DF8CF9CE0980F953044
:101C100070F4845F990B21E030E001C0220F8A95B7
:101C2000EAF78091C402822B8093C40208958D3F0D
:101C300031F48091BD0281608093BD0208958E3F92
:101C400021F48091BD028260F7CF8F3FB9F7809178
:101C5000BD028460F1CFF894E82FE295EF70F0E0D8
:101C600031A1282F2F7081E090E001C0880F2A95C4
:101C7000EAF7982F9095932391A392A1892B82A3A1
:101C8000789408959091900292FF06C0282F2871B1
:101C90002830F9F4877F846093FF06C0282F2871CD
:101CA0002831F1F4877E84612091910220FF06C0E3
:101CB000382F38713830D9F4877F816021FF06C012
:101CC000282F28712831D1F4877E816194FD877E89
:101CD0000895282F24712430F9F68B7F8860DCCF9B
:101CE000282F2471243101F78B7E8861DDCF382FB6
:101CF0003171313019F78E7F8860E0CF282F217144
:101D0000213121F78E7E8861E1CFCF93DF93EC0103
:101D100082389105A9F1D8F58133910509F496C06F
:101D200048F58932910509F48AC08A9709F495C06B
:101D3000C11521E5D20708F0BCC0C11530E5D307B5
:101D400008F014C1C83ED10508F09CC0C03ED105C2
:101D500060F5C83AD10508F087C0C53AD10508F04A
:101D6000FDC0C130D10509F12097F9F0C430D1058B
:101D7000E0F440C08533910509F45AC0C997C1F613
:101D800080919002837089F0C0EED0E00EC0833E57
:101D9000910599F170F4803E910501F1823E910523
:101DA00039F68091900282FD21C0CE01DF91CF9162
:101DB0000895863E910561F1873E910571F1843E5B
:101DC000910509F0B5CF8091910281FFEECF80910E
:101DD0009002C7EED0E084FD0DC0E7CF8091900265
:101DE00080FD12C19091910290FFDFCFC3EED0E051
:101DF00084FFDBCFD0E0C0E0D8CF8091900282FD9D
:101E000006C19091910290FDBFCF84FFCECFF2CF5B
:101E10008091900283FDDDCFC8CF8091900283FD39
:101E2000F9C09091910291FFF0CFC4EED0E0BDCF08
:101E30008091900285FFB9CFC9E2D0E0B6CF809102
:101E4000900285FFB2CFC5E3D0E0AFCF8091900282
:101E500086FFABCFCAE2D0E0A8CF8091900286FF88
:101E6000A4CFC1E3D0E0A1CFCF3BD10518F6C85A2B
:101E7000D0E0CC0FDD1FCB57DE4F0990D881C02DAD
:101E8000D46493CFC11540E2D40758F4C11581E062
:101E9000D80708F08ACFC03FD10508F4ABCFD06592
:101EA00084CFC11590E4D90708F4A4CFDF70D06ABD
:101EB0007CCFC11525E5D20700F5C11534E5D30760
:101EC00008F08AC0C11543E5D40708F071C0C115F8
:101ED00082E5D80708F467C0CE018370992721E016
:101EE00030E002C0220F331F8A95E2F7C695C695EF
:101EF00080E2C89FE001112452C0C11599E5D907BD
:101F0000A8F4C11528E5D20708F06BC0C11536E565
:101F1000D30708F06FCF8C2F0E94420EC82FD0E05D
:101F2000DC2FCC27CC27DF71D0623FCFC1154AE52B
:101F3000D40708F45BC0CE0190568115904208F09A
:101F400059CF8D2F8F710E94420E90E0982F8827D5
:101F500088279F719C012C2BE901E6CFC55AD0E060
:101F6000CE57DE4FC881D0E0D0641FCFCE01E4E071
:101F700096958795EA95E1F783702C2F26952695FF
:101F8000237040E2249F90011124382B8C2F837002
:101F9000C1E0D0E002C0CC0FDD1F8A95E2F7C22B72
:101FA000D32BDC6802CFDC2FCC27C16FD06AFDCEEB
:101FB000CE018370992721E030E002C0220F331F49
:101FC0008A95E2F7C695C69590E2C99FE001112473
:101FD000C22BD32BDA68E9CEDC2FCC27C46FD06AB2
:101FE000E4CEDC2FCC27C06FD06ADFCE8C2F8F7071
:101FF0000E94420E34E0D695C7953A95E1F7CF702E
:102000009C2FEC01D069D1CEC9E3D0E0CECEC2EE98
:10201000D0E0CBCEC6EED0E0C8CE80917702811161
:10202000109277020895809590917602982390936C
:1020300076020895ECE0F2E09191891303C0DF018C
:1020400011971C9292E0E231F907B1F70895ACE0E4
:10205000B2E0EFEF90E02D91821751F0EF3F19F4CD
:10206000211101C0E92F9F5F9630A9F7EF3F09F4D6
:1020700008950E2E000CFF0BE65FFD4F828308953E
:1020800080916B0290913A02981301C008958F5F7E
:102090008770FACF292F953078F5813168F590E077
:1020A00031E1239F800D911D1124682F677023E07B
:1020B000969587952A95E1F7FC01EE0FFF1FE80F33
:1020C000F91FED5EFD4F50E040E080E0219130E0EF
:1020D000062E02C0369527950A94E2F72170332721
:1020E000042E01C0220F0A94EAF7822B4F5F5F4F44
:1020F0004330510559F7089580E00895292F953010
:1021000098F5813188F590E031E1239F800D911D94
:102110001124282F277041E001C0440F2A95EAF7C7
:1021200023E0969587952A95E1F7FC01EE0FFF1FB6
:10213000E80FF91FED5EFD4F30E020E070E05191B7
:10214000DF011197CB01022E02C0969587950A9464
:10215000E2F7817081958527842385278C932F5FF3
:102160003F4F2330310559F7089581FF02C0289A67
:10217000089528980895829590E09C01220F331FBE
:10218000220F331F2C7C95958795959587958373A2
:10219000282B30E0C901880F991F8A7A3595279539
:1021A0002575822B08959FB7F89410923F039FBF27
:1021B00090914E03943009F048C02091E9002F70AF
:1021C0003091EC00932F917030FD90E8922B25E038
:1021D0002093E9002091EB0020FF34C02091EE0015
:1021E00027FF30C020913E03222321F02091E800F8
:1021F00025FF28C010923E0326E03091E80035FF0D
:1022000014C08093F1008091E80085FD27C0809183
:10221000E80080FFFCCF8091E8008E778093E80093
:102220009F709093E90080E0089530914E03343020
:1022300049F43091EB0035FD05C0215041F481E0B7
:1022400080933E039F709093E9008FEF0895EFE92C
:10225000FFE03197F1F700C00000CFCF8FB7F894BF
:1022600021E020933F038FBFDBCF80933B0370932C
:102270003D0360933C0380914E038430F9F48093D6
:10228000E9008FEF9091E800815095FD06C095ED33
:102290009A95F1F700008111F5CF8091E80085FF54
:1022A0000DC050E040E063E070E08BE393E00E94FB
:1022B000A90A8091E8008E778093E8000895BC0118
:1022C00084E00E9435110895BC0183E00E9435111D
:1022D00008959C0184E08093E9009FEF8091E800DD
:1022E000915085FD06C085ED8A95F1F700009111AA
:1022F000F5CF8091E80085FF0CC050E040E066E03B
:1023000070E0C9010E94A90A8091E8008E7780934D
:10231000E8000895CF93DF93EC0181E08093E9001A
:102320008FEF9091E800815095FD06C095ED9A954C
:10233000F1F700008111F5CF8091E80085FF14C00E
:1023400050E040E068E070E0CE010E94A90A809170
:10235000E8008E778093E80088E0FE01A4E4B3E013
:1023600001900D928A95E1F7DF91CF91089581E078
:102370008093E00080E28093D8001092C9008FE142
:102380009EE40197F1F700C0000087E090EBDC01CC
:1023900080935C0390935D03A0935E03B0935F030F
:1023A00088E19CE00FB6F894A895809360000FBE7A
:1023B00090936000FFCF8091240380FD0AC0E4ED7C
:1023C000F2E0118210821282339652E0E23FF5076A
:1023D000C1F76E9A3EB13F7B2EB120644FB7F8949F
:1023E00084ED92E0FC015191CF0168E02EB900002C
:1023F00000C057FF3EB9550F000000C000C000C02C
:102400003EB900C06A9591F7F2E0823F9F0751F70D
:102410004FBF8FE594E00197F1F700C000000895E9
:10242000EF92FF920F931F93CF93DF938C01C4ED34
:10243000D2E0F12CE12CF801948160912603809187
:102440002503F5E0EF16F104ECF49923E9F09E0181
:10245000409127030E944B0C2FEFE21AF20A2396B9
:102460008AE0E816F10439F70E94DB11F801848153
:1024700090E00196817099278483CDB7DEB7E6E0BE
:102480000C94B134992319F39E0140E0E3CFB0E0FE
:10249000A0E0EDE4F2E10C948F34EC014C81042FC8
:1024A00010E09801D8010E94D2359B01AC010E9436
:1024B0009D354B015C01E0E2F0E0E01BF10BA5E58E
:1024C000B0E0AC019B010E949D356B017C019F0136
:1024D000DF010E947A349B01AC010E94A8359B0168
:1024E000AC01280D391D4A1D5B1DC701B6010E94B4
:1024F000B035F22E822F90E039E23F1598F143E09B
:10250000249F9001112435952795122F109594ED55
:10251000C92E92E0D92E00E085E5E82EEF188E2D29
:1025200001FD8F2D9601412F609126030E944B0CD7
:102530000F5F53E0C50ED11C0A3089F70E94DB11F2
:102540009C8181E0992319F0903219F48FEF8093E8
:102550001D0180911D01890F8C83CDB7DEB7ECE0A2
:102560000C94AB3425E530E0A901481B590BCA0196
:102570009A01220F331F280F391F37FFC4CF2F5F57
:102580003F4FC1CF0F931F93CF93DF93C4EDD2E0A2
:10259000FE01118210821282339682E0E23FF80738
:1025A000C1F710E000E08091D202082E000C990BD8
:1025B000081719078CF180911C01082E000C990B4B
:1025C000801791074CF19E014091270360912603EB
:1025D000809125030E944B0C0F5F1F4F23960A30FA
:1025E000110509F70E94DB1180911B019091D20225
:1025F000980F9093D20220911C01280F20931C0168
:10260000121614F499301CF0819580931B01DF9110
:10261000CF911F910F910895198218821A82DCCFF1
:10262000B0E0A0E0E6E1F3E10C949234FC01828199
:10263000DD24DA9480FD02C0DD24D39404ED12E0A1
:10264000D0E0C0E02AE0B22EF8011182108212829E
:1026500094E0E92EF12CC12C8091D1028C0D8B30AD
:10266000C4F16B2D0E943734892F082E000C990B72
:102670008C179D0791F4809127038E9DA0018F9D5B
:10268000500D1124559547955595479598016091A2
:102690002603809125030E944B0CCD0CF1E0EF1A2C
:1026A000F108D1F621960D5F1F4FCA30D10561F6B2
:1026B0000E94DB118091D10291E0D91210C08111EA
:1026C0000CC089E08093D102CDB7DEB7E9E00C946D
:1026D000AE3487FFCACF865FC8CF8150F3CF90E07A
:1026E0000196BE010E945934EDCFEF92FF921F93E5
:1026F000CF93DF93EC0184EDE82E82E0F82E10E01A
:102700008C8197014091270360912603810F0E94DD
:102710004B0C175E83E0E80EF11C1A3F89F70E940C
:10272000DB119A818C8190FF08C08F5F8C83DF91D1
:10273000CF911F91FF90EF9008958150F7CF909126
:10274000240390FF0CC0E4EDF2E0818360834283B8
:10275000339692E0E23FF907C1F70E94DB1108953A
:10276000A3E0B0E0E6EBF3E10C9497348C018091A8
:10277000D30281110AC09E012F5F3F4F4FEF6FEFD1
:102780000E944B0C8A818093D302F80164816130EE
:1027900069F08091D30240E0662361F040E062304E
:1027A00011F44091D30280E060E004C06091D30254
:1027B00040E080E00E949F13F801848190E0019640
:1027C00063E070E00E94593484832396E4E00C9423
:1027D000B334A3E0B0E0EFEEF3E10C9499349091C0
:1027E000240390FF0AC09E012F5F3F4F0E944B0CB5
:1027F0004B8169818A810E949F132396E2E00C94A9
:10280000B534CF93DF93EC01E4E2F3E043816281DE
:102810008C810E94E9138C818F5F8C83DF91CF9133
:102820000895CF93DF93EC01EC81F0E0E752F84F8D
:102830004491E4E2F3E0628181810E94E9138C819A
:102840008F5F8C83DF91CF910895CF93DF93CFEC8F
:10285000D2E060E0CE010E944A352196C11584E0A5
:10286000D807B9F7DF91CF9108951F93CF93DF93E6
:10287000122F8430E0F46530D0F44131C0F4C42F1D
:10288000D0E0CC0FDD1F92E2699FC00DD11D112455
:102890009AEA899FC00DD11D1124632FCE0187961E
:1028A0000E944A35612FCE0188960E944A35DF91F9
:1028B000CF911F910895AF92BF92CF92DF92EF9286
:1028C000FF921F93CF93DF938AE5C82E8FE0D82E17
:1028D000D0E07601C0E014C0F50125913491412F7C
:1028E0006C2F8D2F0E94351482E0A80EB11C1F5F43
:1028F000113191F782E2E80EF11CCF5FC53019F07B
:10290000570110E0E9CFDF5F8AEAC80ED11CD4304E
:1029100001F7DF91CF911F91FF90EF90DF90CF9063
:10292000BF90AF900895CF93C82F6FEF811162E2EF
:1029300083E290E00E944A356FEFC11168E084E2C3
:1029400090E00E944A356FEFC11165E085E290E0AA
:102950000E944A35CF91089580E00E94931460E070
:1029600086E290E00E944A350E945B140E94251482
:1029700081E00E94931408950F931F93CF93DF93E8
:10298000843030F5653020F5413110F5C42FD0E0AA
:10299000CC0FDD1F22E2629FC00DD11D11243AEA47
:1029A000839FC00DD11D1124CE0187960E9436351C
:1029B000082F10E0102F0027CE0188960E94363590
:1029C0009801282BC901DF91CF911F910F91089594
:1029D00090E080E0F8CF462F843040F4753030F43A
:1029E000613120F4672F0E94BC14089590E080E0CC
:1029F0000895CF92DF92FF920F931F93CF93DF93AF
:102A00006C0100915B0380917802082BC7E0D0E055
:102A100010E0FC2EC8010C2E02C0959587950A94F3
:102A2000E2F780FD0CC02197A0F7F12C8F2DDF91EC
:102A3000CF911F910F91FF90DF90CF900895B60135
:102A40008C2F0E94EB140E94850E019761F3EECF4C
:102A5000CF93DF93EC010E94F914BE010E94EB14A6
:102A60000E94850EDF91CF910895FC0180819181B4
:102A70000E94281592959F70963091F058F4925FBD
:102A80009F70923058F4803F19F030F4883E30F453
:102A900081E008959A5FF4CF843FD1F380E00895F8
:102AA000883EB0F3813FD1F7F3CF83E290E00E94FC
:102AB0003635823289F484E290E00E9436358830DF
:102AC00059F485E290E00E94363591E0853009F0B6
:102AD00090E0892F8170089580E0FCCFCF9384E04F
:102AE00090E00E943635C82F82E290E00E94363591
:102AF000982F8C2FCF91089580911E011F928F9354
:102B000080911F011F928F93809120011F928F93BC
:102B1000809121011F928F93809122011F928F93A8
:102B2000809123011F928F9381EC9DE09F938F935F
:102B30000E94500A8DB79EB70E960FB6F8949EBFAE
:102B40000FBE8DBF0895883228F58E3108F072C00F
:102B50008B3041F130F4873009F4CFC080E29FE040
:102B6000E0C0833109F45FC08431C1F782E49FE0A3
:102B70000E94B70980912F03882309F4FEC01092A8
:102B80002F0310922E0310922D0310922C031092FB
:102B90002B0320C08F3409F4C7C0D8F5893231F334
:102BA0008833E1F685E49FE00E94B7090E947C1516
:102BB0001F9281E08F931F9288E08F938EE39EE0B7
:102BC0009F938F930E94500A0F900F900F900F9039
:102BD0000F900F9020912F03222309F4C9C08091F8
:102BE0002B0390912C03009711F485E291E09F93C1
:102BF0008F931F922F938EE09FE09F938F930E945D
:102C0000500A0F900F900F900F900F900F9081E04F
:102C10000895813509F49CC008F49CC0823509F000
:102C20009DCF81E082C084E39FE00E94B7090E94AB
:102C30007C15D0CF8D5180932F03833009F442C08F
:102C400058F48130C1F08230A1F110922F0381E35A
:102C50009FE00E94B7091BC0853009F445C0D8F138
:102C6000863099F78EE191E090932E0380932D03A7
:102C70008DE691E008C083E291E090932E0380936B
:102C80002D0389E291E090932C0380932B03809194
:102C90002F03882309F49ECF1F928F938DE29FE02C
:102CA0009F938F930E94500A0F900F900F900F9058
:102CB00091CF82E291E090932E0380932D0382E3E3
:102CC00091E0E1CF81E291E090932E0380932D0378
:102CD0008EE391E0D8CF80E291E090932E03809331
:102CE0002D038BE491E0CFCF8FE191E090932E0301
:102CF00080932D038AE591E0C6CF81E08093230184
:102D000084E1809322018AE0809321018EE1809307
:102D1000200188E080931F0188E280931E0183E2F6
:102D20009FE00E94B70956CF8AE0E0912D03F09111
:102D30002E033097D1F02081082E000C990B820FC2
:102D4000911D8F3F910541F03CF08FEF808307C0CC
:102D50008FEFEBCF86EFE9CF97FFF8CF108280811E
:102D60001F928F938AE19FE09BCF87E19FE0D9CFAD
:102D70008AE09FE00E94B7094ACF80E00895109250
:102D8000D00280912A0380FF08C080EC97E09F93D7
:102D90008F930E94500A0F900F90089580912A03FC
:102DA00083FF7EC082ED95E00E94B7098091C40246
:102DB0001F928F938DEC95E09F938F930E94500A02
:102DC0008BEC95E00E94B7098091C502282F082E50
:102DD000000C330B3F938F9388EC95E09F938F9378
:102DE0000E94500A86EC95E00E94B7098091C602C5
:102DF000282F082E000C330B3F938F9383EC95E024
:102E00009F938F930E94500A81EC95E00E94B7092E
:102E10008091C702282F082E000C330B3F938F930D
:102E20008EEB95E09F938F930E94500A8CEB95E078
:102E30000E94B7098091C802282F082E000C330B7E
:102E40003F938F9389EB95E09F938F930E94500A55
:102E500086EB95E00E94B7098091BE021F928F9386
:102E600083EB95E09F938F930E94500A81EB95E04E
:102E70000E94B7098091BD021F928F938EEA95E060
:102E80009F938F930E94500A8BEA95E00E94B709A6
:102E90008DB79EB74C960FB6F8949EBF0FBE8DBFF0
:102EA0000E94F00B9C019091C5028091C602982B64
:102EB00021F03093C2022093C1029091C702809109
:102EC000C802982B21F03093C0022093BF02E091FA
:102ED0003203F0913303309749F082E08093C302CC
:102EE0000480F581E02D83EC92E009950895B0E02F
:102EF000A0E0EDE7F7E10C948B34FC0162804480A4
:102F000081E08483E9EDF7E07490E8E5F8E0E4918E
:102F1000C2EFD2E034EDE32E32E0F32E44E2C42ED1
:102F200043E0D42E52E0A52EBB24B39488248A9487
:102F3000912C55245A94E7190E2F10E082E0861543
:102F400030F0809125038883809126038983411086
:102F500016C01B821A8297014A81698188810E946A
:102F60004B0C259683E0E80EF11CCC16DD0631F7FC
:102F70000E94DB11CDB7DEB7E0E10C94A7348B8162
:102F80008823E9F081508B83859DC00111246C81D9
:102F900070E00E944534FB01FF27E752F84F84910F
:102FA000E82FE719E59DC0011124B8010E944534BE
:102FB00080912703689FB00111247A83CCCF0E94AF
:102FC0000C3520912703269521582A9DA0012B9D81
:102FD000500D1124452F5527841795070CF0BBCFB2
:102FE00082E0861588F40E940C35B4010E945934A1
:102FF00088830E940C35209126032695622F70E06D
:103000000E945934280F29831A8280912703893C12
:1030100020F088EC8C838B839ECF8431D8F784E1B9
:10302000F9CFCF92DF92EF92FF926B017C010E9469
:103030003C0CB701A60188E090E00E945C35FF904F
:10304000EF90DF90CF900895A7E0B0E0EAE2F8E1DA
:103050000C948934582E262E342E2F8390912403DD
:1030600090FF46C0E92FE695AE2FB0E0A753BE4FC4
:103070008C918093CF029E7F9230F1F59E012F5F5D
:103080003F4F852D0E944B0C4B8169818A810E94A4
:103090009F135092250320922603309227038F819D
:1030A000882309F48CC060912403709125038091DA
:1030B0002603909127030E94111880912A0380FF14
:1030C00017C0809127031F928F93809126031F9230
:1030D0008F93809125031F928F938FE697E09F93A4
:1030E0008F930E94500A0FB6F894DEBF0FBECDBF7B
:1030F0002796E2E10C94A534823019F4309027032E
:10310000C8CF863019F450902503C3CF8930D9F346
:10311000893109F0BECFE9518E2F81708D838E2FBA
:10312000809581708E83E695F0E0E554F84F949198
:103130009C83692E712C84EDE82E82E0F82ED12C30
:10314000C12C10E000E09AE0892E912C24E9A22EF7
:1031500027E0B22EC601B4010E9445348D81452C72
:1031600081112BC0460E80912A0380FF13C01F924D
:103170009C819F931F928E818F931F924F921F93DA
:103180000F93BF92AF920E94500A0FB6F894DEBF21
:103190000FBECDBF9701432D622D842D0E944B0C95
:1031A0000F5F1F4FC60CD71C93E0E90EF11C0A30CD
:1031B000110581F60E94DB116CCF461AD4CF8091A5
:1031C0002A0380FF95CF1F923F921F922F921F924A
:1031D0005F9288E497E083CFE4E2F3E0438121E16A
:1031E000421B08F440E021E0628181810E942418A2
:1031F0000895E4E2F3E0438121E1420F08F44FEF48
:1032000021E0628181810E9424180895E4E2F3E0C4
:10321000628121E1621B08F460E021E04381818149
:103220000E9424180895E4E2F3E0628121E1620F34
:1032300008F46FEF21E0438181810E9424180895F2
:10324000E4E2F3E0818121E04381628188500E94C1
:1032500024180895E4E2F3E0818121E04381628152
:10326000885F0E942418089580912803882319F00C
:1032700081508093280360912403709125038091ED
:103280002603909127030E94111808958091280326
:10329000833018F48F5F809328036091240370912A
:1032A000250380912603909127030E941118089509
:1032B0009091240390FF40C0917081113EC09260B4
:1032C00090932403662309F43FC060912403709116
:1032D000250380912603909127030E941118809165
:1032E0002A0380FF0FC08091240386951F928F933D
:1032F0008CE297E09F938F930E94500A0F900F905B
:103300000F900F9060912403669570E04BE050E0C1
:1033100080E191E00E941C35892B11F10E94BF16BB
:1033200081E08093CC0220E0409127036091260346
:10333000809125030E94241808958B3210F0946523
:10334000BFCF880F982BBCCF80912A0380FFDACFA4
:103350008091240386951F928F938EE097E0CACFC9
:1033600081E08093D0020E94F00B9093CA02809378
:10337000C90280912A0380FFD3CF85EF96E09F9307
:103380008F930E94500A0F900F90CACF8091240310
:103390008695815009F48AE261E00E9458190895E7
:1033A0008091240386958F5F8B3208F081E061E085
:1033B0000E94581908959091240390FF08C0969593
:1033C000981728F0961718F40E94D019089561E014
:1033D0000E9458190895E4E2F3E083E080831182AB
:1033E0008FEF8283838314826081718182819381D4
:1033F0000E9411180895A4E1B0E0E1E0FAE10C9414
:103400008B348E010F5F1F4F84E1F80111928A9572
:10341000E9F793EBE92E91E0F92E6801AA24A39431
:10342000B12C39EC832E31E0932EF70181917F018D
:103430008F3F09F44FC0F894E82FE295EF70F0E069
:1034400021A18F70A50102C0440F551F8A95E2F794
:10345000CA01922F982B91A392A18095892382A3D0
:10346000789400C0E8EBF1E041E050E060E070E00B
:10347000412C512C320121912F3F09F46EC0A22F13
:10348000A295AF70B0E090968C9190E02F7002C042
:10349000959587952A95E2F780FD5FC0DB01CA010B
:1034A000482A592A6A2A7B2A440F551F661F771F0C
:1034B0008E169F0601F7F701319780818F3F11F03B
:1034C0000E942B0E50EA5A95F1F7F6014082518284
:1034D00062827382F4E0CF0ED11C48EBE41641E027
:1034E000F40609F0A2CF44E150E0B8018CE792E085
:1034F0000E942935FF24F394009709F4F12C892BBD
:1035000081F184E1F801ACE7B2E001900D928A9577
:10351000E1F781E080937B020E94F00B90937A02A6
:10352000809379028091790290917A020E94E10B56
:103530000597D8F0ECE7F2E0A8EAB2E041915191AA
:10354000619171914D935D936D937D9352E0E0395C
:10355000F507A1F710927B0208C080E090E0DC0143
:103560009FCF80917B028111DDCF8F2D6496E0E1AA
:103570000C94A7340F931F93CF93DF93809176021F
:1035800090917502892B80930A029091770299237A
:1035900091F0892B80930A0220E08CE092E0FC01FC
:1035A0003191CF0131112F5FF2E082319F07B9F7DE
:1035B00021110E940D1048E050E06DE672E08AE0B3
:1035C00092E00E942935892B09F441C088E0EAE0A5
:1035D000F2E0ADE6B2E001900D928A95E1F7E0915C
:1035E0003203F0913303309791F10280F381E02DA3
:1035F0008AE092E0099580912A0382FF28C080FF2B
:1036000004C087E493E00E94B709D0E0C0E001E481
:1036100013E080912A0380FF0EC0FE01E65FFD4F9C
:1036200080811F928F931F930F930E94500A0F90D7
:103630000F900F900F902196C830D10551F78091CF
:103640002A0380FF04C08FE393E00E94B709DF9153
:10365000CF911F910F91089590E080E00E94120C8D
:1036600090E080E00E94FC0B109275020E94BA1A52
:1036700086E0E3ECF2E0DF011D928A95E9F7109213
:10368000BE021092BC021092BD020E94CE16089596
:1036900080935B030E942C1B089580915B03982FFD
:1036A0009670963021F488600E94481B0895877FA9
:1036B000FBCF21E030E001C0220F8A95EAF7209588
:1036C00080915B0382230E94481B089590916C02B5
:1036D0008095892380936C02282F277091F4282FDE
:1036E000082E000C330B9217130659F0909191029B
:1036F00092FF07C08595859585950E94591B10926C
:103700006C020895CF93DF93D82FC0919102C2FB32
:10371000882780F98D1711F1D0FBC2F9C09391026F
:103720006091900284E090E00E944A356C2F82E222
:1037300090E00E944A3582E00E94661B80912A0335
:1037400080FF0CC01F92DF938AE293E09F938F93D8
:103750000E94500A0F900F900F900F90DF91CF9121
:10376000089521E030E001C0220F8A95EAF78091A8
:103770005B03822B0E94481B0895809378020E946D
:103780002C1B0895882321F00E9413100E94BA1A5E
:103790000895882339F090917602982B90937602C1
:1037A0000E94BA1A0895882309F455C0823879F422
:1037B0000E94280C81FF4FC089E30E9427100E94BD
:1037C000BA1A89E30E941A100E94BA1A089583381F
:1037D00059F40E94280C80FF3EC083E50E94271008
:1037E0000E94BA1A83E5EECF843859F40E94280C5F
:1037F00082FF31C087E40E9427100E94BA1A87E432
:10380000E1CF9CEF980F913AE8F290E2980F983050
:1038100050F4877091E001C0990F8A95EAF7892FDB
:103820000E941310D1CF9BE5980F933028F490E0BD
:1038300080E00E94120C089598E5980F973128F4C3
:1038400090E080E00E94FC0B0895803F20F00E94F1
:10385000E10C0E94CE16089568EE7EEF90E080E0C5
:103860000E94683560E082E090E00E944A3560E0A6
:1038700083E090E00E944A351092780260E084E094
:1038800090E00E944A3564E082E290E00E944A356E
:1038900060E085E090E00E944A3560E086E090E0DC
:1038A0000E944A356FEF87E090E00E944A3540E081
:1038B00050E0BA0188E090E00E945C3560E08DE065
:1038C00090E00E944A3540E050E0BA0188E190E083
:1038D0000E945C3560E087E190E00E944A3540E05C
:1038E00050E0BA018CE190E00E945C3570E060E04D
:1038F00080E290E00E94683540E050E0BA0188E143
:1039000090E00E945C3580E00E9493140E94AC1409
:1039100040E050E0BA018FE090E00E945C3540E06A
:1039200050E0BA0183E190E00E945C350895109266
:103930007602ECE0F2E086E0DF011D928A95E9F77D
:103940000E942C1B0895AAE2B0E0E9EAFCE10C9485
:10395000983480E593E02091F100DC012D93CD01B6
:10396000B3E088359B07B9F780915103833009F4A0
:1039700072C0B8F4813009F449C0823009F4B3C090
:103980008091E80083FF91C2809150039091510390
:103990009A3008F08AC2E92FF0E0ED51FA4C0C940D
:1039A0006D348A3009F48EC08B3009F471C08930CF
:1039B00039F780915003813219F780915403909127
:1039C0005503009711F00297D9F68091E800877FA0
:1039D0008093E8008091E80082FF38C09091F30066
:1039E0008091F200029731F48091F100813011F062
:1039F000863021F48091F100809343038091E800A8
:103A00008B778093E8000E94D30ABACF809150034D
:103A1000813A09F0B5CF8091E800877F8093E80074
:103A20008091540390915503892B61F468E084E4FC
:103A300093E070E00E947F0B8091E8008B77809389
:103A4000E8009ECF60E090E080E0F3CF80914E03ED
:103A50008111C0CF95CF80915003813A09F090CF6A
:103A60008091540390915503892B09F089CF80915F
:103A7000E800877F8093E8008091E80080FFFCCF1A
:103A8000809124018093F1008091E8008E77B9CF76
:103A900080915003813209F073CF8091540390914B
:103AA0005503892B09F06CCF8091E800877F8093C4
:103AB000E8000E94D30A80915203809324010E945F
:103AC000971C5ECF80915003813209F059CF8091CD
:103AD000E800877F8093E8000E94D30A8091530317
:103AE000809342034DCF80915003813A09F048CF33
:103AF0008091E800877F8093E8008091E80080FF54
:103B0000FCCF80914203BECF803899F0823809F013
:103B1000CCC1809154038F70873008F0C6C1809368
:103B2000E9008091EB0085FB882780F91092E9007D
:103B300006C080914C0390914D0391118260909149
:103B4000E800977F9093E8008093F1001092F100D5
:103B50008091E8008E77A5C1882309F493C1823053
:103B600009F0A3C180915203811196C18091540341
:103B70008F702FEF280F263008F097C18093E9004F
:103B80002091EB0020FF88C1933031F48091EB004D
:103B900080628093EB0080C19091EB0090619093E4
:103BA000EB0021E030E001C0220F8A95EAF7209374
:103BB000EA001092EA008091EB008860EACF811160
:103BC00074C1109152031F778091E3008078812B9C
:103BD0008093E3008091E800877F8093E8000E9453
:103BE000D30A8091E80080FFFCCF8091E3008068D9
:103BF0008093E30082E0111183E080934E0355C16E
:103C00008058823008F051C1209152033091530303
:103C10002C3DE3E03E07A1F583E08A838AE28983B5
:103C20004FB7F894DE01139620E03EE051E2E32F17
:103C3000F0E050935700E49120FF03C0E295EF704D
:103C40003F5FEF708E2F90E0EA30C0F0C7968D9303
:103C50009D932F5F243159F74FBF8091E800877FF4
:103C60008093E8006AE270E0CE0101960E947F0B2B
:103C70008091E8008B778093E80017C1C096E7CF6A
:103C80008091540390915503432F5527433051059C
:103C900009F44AC078F54130510509F47AC08BE740
:103CA00090E0E6E1F2E14230510509F0FEC02091DA
:103CB000E800277F2093E8002091560330915703B6
:103CC0008217930708F49C0140E02115310509F0A3
:103CD00065C0411163C08091E80082FDC9CF809129
:103CE0004E03882329F2853019F28091E80083FF82
:103CF000F2CFBECF4132510509F43CC042325105EA
:103D000009F0D3C08430910508F0CFC0FC01EE0F5C
:103D1000FF1FE850FE4F0190F081E02D8C509E4F28
:103D2000DC018C9190E01AC0332721303105D1F0AD
:103D30002115310561F02230310509F0B6C0E3EA02
:103D4000F2E1E4918E2F90E0E3EAF2E107C0EDEDBD
:103D5000F2E1E4918E2F90E0EDEDF2E1009709F4AD
:103D6000A4C0A5CFEFEBF2E1E4918E2F90E0EFEB52
:103D7000F2E1F4CF8430910508F097C0880F991FC5
:103D8000FC01E050FE4F0190F081E02D89E090E0D1
:103D90008ECF82E190E0E1E9F2E189CF80914E039C
:103DA000882309F465CF853009F462CF8091E8005B
:103DB00083FD5ECF8091E80082FD8DCF8091E80089
:103DC00080FF83CF9091F3008091F200211531059F
:103DD00019F08830910550F041E0089709F040E073
:103DE0008091E8008E778093E8006FCF44914093F4
:103DF000F1003196215031090196E8CF803809F061
:103E000054C08091E800877F8093E80080914F0341
:103E10008093F1009DCE811148C010915203123061
:103E200008F043C08091E800877F8093E8001093FA
:103E30004F030E94D30A112311F084E005C0809142
:103E4000E30087FDFACF81E080934E0342E061EC0E
:103E500081E00E94F20A42E261EC84E00E94F20AF0
:103E600042E261EC82E00E94F20A42E260EC83E00E
:103E70000E94F20A42E261EC85E00E94F20A80911F
:103E80004E0313C080915203813079F481E0933066
:103E900009F080E080934D031092E9008091E800E2
:103EA000877F8093E8000E94D30A8091E80083FF17
:103EB0000AC08091E800877F8093E8008091EB0042
:103EC00080628093EB00AA96E3E00C94B434CF9325
:103ED000C82F1F928F9385E59FE09F938F930E9439
:103EE000500A81E001C0880FCA95EAF70E94BD1B05
:103EF0000E94971C0F900F900F900F90CF910895F4
:103F0000CF92DF92EF92FF92CF93DF938B3109F440
:103F10000FC108F0A3C08B3009F4C9C008F081C0FC
:103F2000863009F4D7C048F4853009F4A5C082E290
:103F30009DE00E94B70980E0DDC0873009F4E1C050
:103F40008830A9F783E090E00E9436351F928F9366
:103F500087E09AE09F938F930E94500A82E090E05E
:103F60000E94363583FB992790F91F929F9382FB1D
:103F7000992790F91F929F9381FB992790F91F929F
:103F80009F93982F91701F929F931F928F938EEB08
:103F900099E09F938F930E94500A0E946E1587FBB1
:103FA000222720F91F922F9386FB222720F91F92A8
:103FB0002F9385FB222720F91F922F9384FB222722
:103FC00020F91F922F9383FB222720F91F922F9312
:103FD00082FB222720F91F922F9391FB222720F9A1
:103FE0001F922F93292F21701F922F9381FB22273D
:103FF00020F91F922F93282F21701F922F939F93A8
:104000008F9389ED98E09F938F930E94500A8DB70C
:104010009EB788960FB6F8949EBF0FBE8DBF81E005
:1040200069C0803109F49CC080F48E3009F07FCFE4
:1040300090912A03892F8B7F92FF846080932A03BB
:1040400082FF8BC08DE49DE07FC0863109F498C06B
:10405000893109F06CCF8EEE9BE02BC08A3299F14A
:10406000E0F4873261F128F48E3108F460CF8D518D
:1040700027C0893209F05BCF80E99DE00E94B70933
:104080000E94971C9FEF24E38CE0915020408040D9
:10409000E1F700C000000E94B711833468F48A334E
:1040A00008F098C0853359F0883309F040CF84E296
:1040B0009AE00E94B709B3CF833409F038CF80E08B
:1040C0000E94671FACCF80EB9DE00E94B7090E9461
:1040D0002C1CA5CF80912A03807F80932A0387EC34
:1040E0009BE00E94B7098CEA9DE00E94B70981E03D
:1040F00080932903DF91CF91FF90EF90DF90CF90D5
:10410000089590912A03892F8E7F90FF816080937C
:104110002A0380FF03C084E89DE0CBCF87E79DE0C2
:104120000E94B70980912A03817F80932A0377CF69
:1041300090912A03892F8D7F91FF826080932A03BB
:1041400081FF08C08AE69DE00E94B70980912A039A
:104150008160EBCF8CE59DE0ACCF8DE39DE0A9CFF6
:1041600090912A03892F877F93FF886080932A0389
:1041700083FF03C081E39DE0E7CF84E29DE099CF18
:104180008FB7F894C0903703D0903803E09039038C
:10419000F0903A038FBFD0914203C09124010E9456
:1041A000280CFF92EF92DF92CF921F92DF931F9223
:1041B000CF931F928F9387EB9CE09F938F930E94E6
:1041C000500A8DB79EB70C960FB6F8949EBF0FBEDF
:1041D0008DBF25CF895374CFCF93C82F8823C9F0C3
:1041E0008238C9F40E94280C81FD13C089E30E9423
:1041F00027100E94BA1A2FEF81EE94E021508040E0
:104200009040E1F700C0000089E30E941A100E946C
:10421000BA1ACF9108958338A1F40E94280C80FD2A
:10422000F8CF83E50E9427100E94BA1A2FEF81EE83
:1042300094E0215080409040E1F700C0000083E509
:10424000E4CF8438A1F40E94280C82FDE2CF87E4F9
:104250000E9427100E94BA1A2FEF81EE94E021509D
:1042600080409040E1F700C0000087E4CECF8CEFA3
:104270008C0F813A08F051C0809129038130F9F008
:10428000882399F0823009F444C010922903ECE0AD
:10429000F2E08191C81709F474C022E0E231F2071C
:1042A000C1F78C2F0E942710B2CF80917602823204
:1042B00071F78C2F0E94801F8111ABCFE8CF8091C6
:1042C00076028232B1F3C431C9F048F4CB3059F0F0
:1042D000C031C1F084E293E00E94B70911C0C93235
:1042E00069F0C833B9F787EC9BE00E94B70986E212
:1042F00093E00E94B70981E08170DECF109229031C
:1043000080E0FACF82E08093290388E30E94A3151E
:10431000F2CF8C2F0E94A3157CCF80E28C0F8830C7
:1043200068F4C77021E030E001C0220FCA95EAF7B7
:1043300080917602822B8093760269CFEBE5EC0FB9
:10434000E33040F4F0E0EE57FE4F808190E00E94B1
:10435000120C5FCFE8E5EC0FE73150F4F0E0EE0F20
:10436000FF1FEB57FE4F808191810E94FC0B51CFC4
:10437000C03F08F44ECF8C2F0E94D10D0E94CE1664
:1043800048CF8C2F0E941A100E94BA1A8ACF1F930E
:10439000CF93DF93182FD0E0C0E0893311F4C0E54C
:1043A000D0E0812F0E94EC20209739F4812F0E94C9
:1043B000D31BDF91CF911F9108958FE99FE0019763
:1043C000F1F700C000002197EFCF0F931F93CF9319
:1043D000DF93C62FD42F022FFC0182818823A9F0FE
:1043E00060935A030E94F00B9093590380935803F3
:1043F000C77081E001C0880FCA95EAF70E94C91B07
:10440000DF91CF911F910F91089580915A03681306
:1044100032C080915803909159030E94E10B883C6F
:10442000910548F510E21D0FCD17B9F080E28C0F11
:10443000883040F4C77081E001C0880FCA95EAF760
:104440000E94C21B183048F481E09D2F977001C074
:10445000880F9A95EAF70E94C91B802F0E94C721F6
:10446000183070F6D77081E001C0880FDA95EAF74E
:104470000E94C21BC5CFC77081E001C0880FCA95DA
:10448000EAF7F6CF0E94971C2FEF84E39CE02150BF
:1044900080409040E1F700C0000088E19CE00FB64A
:1044A000F894A895809360000FBE90936000FFCFB2
:1044B000A5E0B0E0EEE5F2E20C948A348C01FC0158
:1044C00083819481892B31F08081918189238F3F71
:1044D00009F0B8C52596E1E10C94A6340E94F914C0
:1044E000F82E682F89819A810E947E1069817A81D5
:1044F0008F2D0E94EB147C01F8018281882309F43E
:1045000094C5970122513F452031310508F060C51F
:104510008FEF93E00E943635811128C0FEEEEF0E3A
:104520005FEC852E52E0952EE11032C01C821B827A
:10453000442443944AE0342E74018FEFE81AF80AB9
:10454000C4010E94363589831A82882379F09FEF4F
:10455000980F933058F58A83498292E0890E911C16
:10456000C7010E9436358B83811121C080916C0276
:10457000877009F4AFCFF8018281882309F4AACFAC
:104580008091910282FFA6CF82E00E94661BA2CF9B
:10459000811424E0920651F3C4010E943635811142
:1045A00001C0EA943FEF831A930ABECF4701FE0190
:1045B00031967F01F7012081222309F4BDCF2130FC
:1045C00009F047C091818281913031F4F2E0EF0E21
:1045D000F11C0E94C72107C0923049F422E0E20E8C
:1045E000F11C0E94EC203FEFE31AF30AE3CF933073
:1045F00031F432E0E30EF11C0E94D31BF4CF94306F
:1046000021F08FEFE81AF80AEECF92E0E90EF11CE4
:1046100030E020E0B7016F5F7F4FF70141818053A9
:10462000990B8A30910550F021503109E0F28FE961
:104630009FE00197F1F700C00000F6CF329EF00135
:10464000339EF00D11249C012E0F3F1F842F7B0100
:10465000E1CFE22FF0E0E552FE4F5490822F869595
:104660008695869590E0FC01E553FE4F6490277097
:10467000712C022E02C0759467940A94E2F7E1E06F
:104680006E227724FC01E554FE4FA490B12C022E3B
:1046900002C0B594A7940A94E2F7F1E0AF22BB24DC
:1046A000FC01E555FE4FC490D12C02C0D594C794AF
:1046B0002A95E2F721E0C222DD246114710419F089
:1046C00081EE0E94EC20A114B10419F086EE0E9444
:1046D000EC20852D0E94C721A114B10419F086EEAB
:1046E0000E94D31B6114710419F081EE0E94D31B48
:1046F000C114D10409F477CF8CE26BCF81E00E9422
:10470000B11B0E944D1B32CF81E00E94591BF9CF93
:1047100082E0F5CF95EFE9169CE5F90609F46CC047
:1047200008F466C027E245EE66EEF6EFEF16FCE50C
:10473000FF0609F476C4882309F495C410925A033D
:1047400023E0E2162DE5F20608F05DC03AEFE3162D
:104750003CE5F30630F4C70182509C45449708F0CD
:104760005EC00E946E159093910280939002E1E1E9
:10477000EE16ECE5FE0609F436C108F0A4C029E007
:10478000E2162CE5F20609F41CC108F06DC085E0C4
:10479000E8168CE5F80609F408C108F056C0E3E015
:1047A000EE16ECE5FE0609F4F6C008F0FAC08091BA
:1047B0009002816022E0E2162CE5F20609F4EEC0D8
:1047C00060919002F090910284E090E00E944A355E
:1047D0006F2D82E290E00E944A350E94971CC6CE5F
:1047E00027E245EE65EE1DC426E241EE60EE19C4F7
:1047F00027E245EE64EE15C426E241EE62EE11C4F6
:1048000028E241E0EFCF81E6E8168DE5F80609F4ED
:10481000A8CF95EAE9169DE5F90609F4A2CF36E19D
:10482000E3163CE5F30609F007C5809176028A7A23
:1048300091E009F490E090931202811102C189E2A3
:104840000E9427100E94BA1A91CE80919002806235
:1048500037E0E3163CE5F30609F4A0C008F4ADC068
:104860008091900280649AC0809190028B7F9DE03D
:10487000E9169CE5F90609F491C0B0F48091900224
:104880008E7FFBE0EF16FCE5FF0609F487C0809100
:1048900090028C602CE0E2162CE5F20608F47EC053
:1048A000809190028D7F7AC0809190028F7E3FE050
:1048B000E3163CE5F30609F471C008F488C0809162
:1048C00090028F7D6BC09DEFE9169CE5F90609F417
:1048D00086C078F5F5E1EF16FCE5FF0609F491C016
:1048E000A0F480919002837F33E1E3163CE5F30668
:1048F00009F454C008F47BC00E94971C9091900268
:10490000892F97FB87F9805849C09BEFE9169CE5F2
:10491000F90609F44EC008F05EC0809191028160F2
:10492000FAEFEF16FCE5FF0609F04ACF80939102FB
:1049300047CF21E0E2162DE5F20609F46EC0B8F487
:104940008FEFE8168CE5F80609F457C080919102C4
:104950008360E1149DE5F90648F380919102982F58
:10496000909591708E7F892B90FB81F9DFCFE1E6E6
:10497000EE16EDE5FE0609F456C0F5EAEF16FDE584
:10498000FF0609F457C022E0E2162DE5F20609F011
:1049900017CF60E043C080919002826080939002C4
:1049A0000FCF809190028460F9CF8091900288604F
:1049B000F5CF809191028260B9CF809190028061A1
:1049C000EDCF0E94971C809190028068E7CF809184
:1049D0009002877FE3CF809191028E7FA7CF809155
:1049E00091028D7FA3CF809190028F7BD7CF0E94C1
:1049F000971C809190028F77D1CF809191028C7F0C
:104A000095CF8091900282FB992790F921E092271F
:104A100090FB82F990FB83F9C1CF61E08EE090E0DA
:104A20000E944A35CDCE90919002892F8F7E94FFBF
:104A30008061B4CF90919002892F8E7F90FF81602A
:104A4000ADCF85E3FDCE80911202811104C089E2D1
:104A50000E941A10F7CE85E3FBCF81608093240378
:104A600080912A0380FF0DC01F9281E08F9383E91C
:104A700092E09F938F930E94500A0F900F900F9097
:104A80000F908091240361E086950E9458196ECDA5
:104A900046EC59E160ED79E10E94350C67CD40EDBF
:104AA00059E166EC79E1F8CF4AE259E160E279E157
:104AB000F3CF46E059E163E179E1EECF4CEE58E106
:104AC00069EF78E1E9CF49EF58E16CEE78E1E4CFA6
:104AD00046E459E164E379E1DFCF61E081E0D5CFDD
:104AE00065E082E00E94DB1941CD68E086E0FACF04
:104AF00064E18FE0F7CF67E185E1F4CF62E289E11D
:104B0000F1CF61E083E2C1CF90912A03892F8E7F9C
:104B100090FF816080932A0380FF05C083E193E0CA
:104B20000E94B70923CD81E093E0FACF0E942C1CAC
:104B30000E9442228091910282FB882780F991E0B5
:104B400089270E94821BF8018281E080F1808823FE
:104B500009F445C0C7010E94F914D82E682FC70177
:104B60000E947E10B7018D2D0E94EB140E94850ECD
:104B70007C01882EF801D280B580B2943FE0B32248
:104B800080916C028770C1F0AD2CDD20B1F08F2DCB
:104B9000807F803421F080E28E0D883068F0809133
:104BA000910282FF09C082E00E94661B80916C0224
:104BB0008770AA24A3948111A12C9F2C92942FE09A
:104BC0009222FBE0F91508F479C0E92DF0E0E351F9
:104BD000FA4C0C946D3481E0B4CF80E0B2CFC701C1
:104BE0000E944A10D82EBECF2F2D2F70C22E8F2D8F
:104BF000807F19F0C29490EFC922DD20B9F0CC205B
:104C000069F080E28E0D883010F0811009C080912B
:104C10007602C82AC09276020E94BA1A8E2D4CC023
:104C200080917502C82AC0927502F6CF8E2D0E941F
:104C3000D31BCC2009F442C080E28E0D883010F0E6
:104C4000811004C08C2D0E94131006C0C094809166
:104C50007502C822C09275020E94BA1A2FC03F2D59
:104C60003F70C32E8F2D807F803219F0C29480EF69
:104C7000C822882089F081E0881609F46AC0DD2006
:104C800009F474C0BB2009F46AC0F801858180FF73
:104C9000C5CF8F70858363C02091910222FD37C0FC
:104CA000DD2079F1CC2039F080917602C82AC092BB
:104CB00076020E94BA1A80E00E94EC20292D28502A
:104CC000330B2430310520F40E94280C0E94B510CB
:104CD000AA2009F4FFCB80916C0280FDFBCBF80188
:104CE00012828595859585950E94B11BC8010E9409
:104CF000582280916C028595859585950E94591B57
:104D0000E9CB80E00E94D31BCC20C1F29BCFDD20F9
:104D100099F0909177028C2D892BB11003C00E94DD
:104D2000C91BCCCFE1E0BE12FACF22FFC7CF981744
:104D300029F280937702C2CFB11006C00E940D10F5
:104D40008C2D0E94C21BBACFF1E0BF1609F4B6CF7A
:104D5000F5CFDD2031F025E02B1508F4AFCF8C2DF9
:104D6000DECF34E03B1508F4A9CFEACFBB2041F3F6
:104D7000F9E38F1209C02FEF37EE83E02150304066
:104D80008040E1F700C000008E2D0E94D31B96CF1B
:104D90008F2D86958695837061F0813009F08ECFD6
:104DA000C7019370D11002C090E080E00E94FC0B1C
:104DB00085CFC7019370D11002C090E080E00E94BF
:104DC000120C7CCF8E2DDD2029F00E94D10D0E9487
:104DD000CE1674CF0E94E10CFACF8F2D837091F51F
:104DE000D1106CCF4E2D429546954770440F440F1D
:104DF0008E2D8F70042E01C0880F0A94EAF72E2D95
:104E00002071E4FE07C02FE030E001C0220F4A9578
:104E1000EAF720953F2D369536953370323069F09C
:104E200050F440917802313029F0822B84230E9483
:104E3000BD1B44CF842B822BFACF282B8091780284
:104E40008227F5CF8695DD2011F08F2D8170882384
:104E500009F434CF4E2D429546954770440F440FC8
:104E60008E2D8F70042E01C0880F0A94EAF72E2D24
:104E70002071E4FE07C02FE030E001C0220F4A9508
:104E8000EAF720953F2D369536953370323069F02C
:104E900050F440915B03313029F0822B84230E942F
:104EA000481B0CCF842B822BFACF282B80915B03DD
:104EB0008227F5CF9F2D9F70F92EDD2029F0892FB5
:104EC0000E94B11B8E2D2BCF8E2D0E94C21B8F2DC9
:104ED0000E94591BF3CE8E2DE2EF8E16B1F1E8152C
:104EE00070F0F0EF8F16D1F021EF821691F0DD20F7
:104EF00009F45EC0B11092CE8F2D8F712AC033EFAE
:104F0000831651F194EF8912F2CF8091910282FDC4
:104F10002FC08F2D8F71DD20D9F21BC0DD2081F0D5
:104F2000E4E0EB1508F4CACE2F2D2F7181E090E05C
:104F300001C0880F2A95EAF790915B038927AFCFCC
:104F4000F5E0FB1508F4BACEEFCF8F2D8F71D1109D
:104F5000BFCF0E94B11BB2CE80E0DD2009F49FCF0D
:104F60009F2D9F7181E001C0880F9A95EAF797CF36
:104F7000DD2099F02F2D2F71F22E822F0E94B11B70
:104F80008091910282FF07C038E0F39EC001112496
:104F9000836080936C028F2DDCCF81E00E94661BC2
:104FA00081E08B1508F08ACE82E00E94661B86CED7
:104FB000BB2059F0893309F0E7CE9FEFE7EEF3E02D
:104FC0009150E040F040E1F7DDCE8F2D8F7180CF22
:104FD000F0E1EF16FFE5FF0609F490CB21E1E216C0
:104FE0002FE5F20609F494CB93EFE9169CE5F90658
:104FF00009F4FACB08F08ECBF8EDEF16FCE5FF06CE
:1050000009F4EECB29EDE2162CE5F20609F4F8CB13
:1050100037EDE3163CE5F30609F08DCB26E241EED1
:1050200061EEC8010E94E521A1CA30E1E3163FE527
:10503000F30609F469CB91E1E9169FE5F906A1F6BB
:1050400082E063CB85E0DE01119601900D928A9596
:10505000E1F7F801228189819A8121113FCA0E94DA
:105060004A10F82E43CAF6E1EF16FCE5FF0609F4F4
:10507000EACC8091760282722CECE2162CE5F206E4
:1050800009F426CD08F096C096ECE9169CE5F906E1
:1050900009F40ACD08F065C0F3ECEF16FCE5FF0655
:1050A00009F4F6CC08F04CC032ECE3163CE5F3060C
:1050B00009F049CD80912A0380FF10C0809124031C
:1050C000809581701F928F938AEC92E09F938F93CB
:1050D0000E94500A0F900F900F900F908091240320
:1050E00080FFBBCC8E7F809324036091240370915A
:1050F000250380912603909127030E941118809127
:105100002A0380FF0FC08091240381701F928F9328
:105110008BE592E09F938F930E94500A0F900F901F
:105120000F900F900E94BF168FEF90E7E2E0815042
:105130009040E040E1F700C000000E94DB1116CA79
:1051400094ECE9169CE5F90609F4A9CC40E259E192
:105150006AE279E1E5ECEE16ECE5FE0609F49CCC9A
:10516000F2CCF9ECEF16FCE5FF0609F4A7CC88F4C5
:1051700037ECE3163CE5F30609F49BCC43E159E137
:1051800066E079E198ECE9169CE5F90609F484CC2F
:10519000DACCEAECEE16ECE5FE0609F494CC44E336
:1051A00059E166E479E1FBECEF16FCE5FF0609F452
:1051B00073CCC9CC21EDE2162CE5F20609F498CCAB
:1051C000B8F48EECE8168CE5F80609F489CC08F4FE
:1051D00084CCEFECEE16ECE5FE0609F486CC6EE02E
:1051E00089E0F0EDEF16FCE5FF0609F47BCCABCCD3
:1051F00024EDE2162CE5F20609F480CC78F482ED79
:10520000E8168CE5F80609F476CC61E088E193EDC8
:10521000E9169CE5F90609F438CC95CCE5EDEE16D7
:10522000ECE5FE0609F46DCC6AE285E2FDE5EF16D9
:10523000FF0609F457CC87CC2AE5E2162DE5F206E5
:1052400009F4C9CCF0F481E0E8168CE5F80609F41D
:105250005BCC9EEDE9169CE5F90609F467CCE114F8
:10526000ECE5FE0609F06FCC0E94971CFFEF24E3EB
:105270003CE0F15020403040E1F700C000000E94C7
:10528000B711FCE5EF16FDE5FF0609F453CC08F471
:10529000A4CC37EAE3163DE5F30609F449CC53CC38
:1052A0001F93CF93DF9380913902807F09F049C02B
:1052B00080913602882309F444C080916B02D0911A
:1052C0003A026091340270913502A0913702B09198
:1052D0003802C62FC72316E0D81799F190E010972F
:1052E00011F0CF3F19F401968770F6CF189F900107
:1052F000199F300D1124F901E55CFD4F41814713E1
:10530000F2CF40814613EFCF42814111ECCF438170
:1053100054814A1B5B0B483C510528F780913902A8
:105320008F70806180933902F901E05CFD4F8081CC
:105330008F708061808384E392E00E9458220E94F3
:105340004010DF91CF911F910895A1E1B0E0EBEA09
:10535000F9E20C9491348C0185E0F801DE011D9690
:1053600001900D928A95E1F7F801E28084E3A82E7E
:1053700082E0B82E60913702709138026115710594
:1053800009F426C19091340240913502892F84237B
:105390008F3F09F41DC120813181C380D480F090FA
:1053A0003602F601E61BF70BFF2009F4DCC0809102
:1053B0003902582F507FE83CF10508F09FC0511189
:1053C0006BC0FE2C431314C0921312C0E11010C026
:1053D0008F70806180933902C5010E9458228091AC
:1053E0003902F80185838F2D6196EAE00C94AD3483
:1053F000C114D10429F0822F83238F3F09F003C108
:1054000080E0F82FF170DF2E80FF3CC080916B02AE
:1054100040913A0256E0841315C02D873E878D8552
:105420009E850E942815292F22952F702230F0F09A
:10543000243018F59F70F1F0F8019581907FD1F438
:10544000D12C1EC090E0589FF001599FF00D1124FF
:10545000E55CFD4F6181361306C06081261303C0F1
:105460006281E6120FC001968770D5CF9F7011F050
:10547000882331F3805E883018F3C8010E945822D7
:10548000FD2CB1CFEE2009F4AECF809139028160BE
:1054900080933902F12CA7CF431306C0921304C0A6
:1054A000F801EE2009F479C0C8010E94351588235F
:1054B00009F1EE20F9F080913902803270F02091EC
:1054C00034023091350238872F831986DB86CA86ED
:1054D0008C87CE0107960E94582286E0F801A4E34B
:1054E000B2E001900D928A95E1F70E945029FF24C5
:1054F000F39479CFC8010E945822F9CF51110AC004
:1055000084E392E00E94582286E0F50111928A9588
:10551000E9F7C0CF43130FC092130DC0E1100BC0C9
:10552000F8018583C8010E94582286E0F501119296
:105530008A95E9F758CFC8010E9435158823D1F222
:10554000EE20C1F280913902803238F2209134028B
:10555000309135023A8329831B82DD82CC828E838F
:10556000CE010196B8CFE83CF105F8F6FE2CEE200E
:1055700009F243131FC092131DC08091390280FDB0
:1055800010C0982F907F69F0F8018583903F31F02B
:10559000982F907F905F8F70892B8583C8010E9420
:1055A000582286E0F801A4E3B2E001900D928A95BA
:1055B000E1F719CFC8010E94351581118ECF809176
:1055C0003902816080933902C8010E9458220BCFB2
:1055D000EE2009F48FCFC8010E943515F82E8823DC
:1055E00009F488CF86E0F801A4E3B2E001900D92BF
:1055F0008A95E1F780913402909135020E94281536
:105600000E945029F0CE81E08E25FBCEA7E1B0E0CC
:10561000ECE0FBE20C9498344B8B5C8B6D8B7E8BB7
:105620008F8B6111109275021A8A198A85E0FE012A
:105630007396DE011D9601900D928A95E1F786E042
:10564000FE013D96DE01179601900D928A95E1F7D5
:10565000CE0107960E94A529882359F016E0809173
:105660006B0290913A02891343C06796E3E00C9471
:10567000B43486E0FE013796DE01119601900D925A
:105680008A95E1F78A859B85892B41F38F819885DF
:1056900089238F3F19F320913A0230E0C901019626
:1056A0008770992740916B024817190671F40E9480
:1056B000971C10923A0210926B0286E0E4E3F2E04B
:1056C000DF011D928A95E9F7C9CF96E0929FD0013C
:1056D000939FB00D1124A55CBD4FFE013196019042
:1056E0000D929A95E1F780933A020E944010B6CF4E
:1056F000819FC0011124855C9D4F0E94A5298823AC
:1057000009F4B3CF80916B0290E0019687709927DE
:1057100080936B02A4CF90E080E00E944435883EE5
:105720009E4F19F40E945515089580E008951F9228
:105730000F920FB60F9211242F933F934F935F93C5
:105740006F937F938F939F93AF93BF93CF93DF9389
:10575000EF93FF93D091E900DF708091EC00C82FA8
:10576000C17080FDC0E81092E9008091F000877F51
:105770008093F00078940E94A31C1092E90080911D
:10578000F00088608093F000CD2BCF70C093E900CB
:10579000FF91EF91DF91CF91BF91AF919F918F9149
:1057A0007F916F915F914F913F912F910F900FBE1D
:1057B0000F901F9018951F920F920FB60F92112401
:1057C0002F933F934F935F936F937F938F939F9309
:1057D000AF93BF93EF93FF938091E10082FF15C0D9
:1057E0008091E20082FF11C08091E1008B7F809365
:1057F000E100209140032F5F822F62E30E942B344F
:10580000992309F4C0C0209340038091DA0080FFFF
:1058100028C08091D80080FF24C08091DA008E7F5C
:105820008093DA008091D90080FFE3C080E189BDD8
:1058300082E189BD09B400FEFDCF81E080934E0373
:1058400082E092E10E94B70980914103811109C071
:105850000E94590A0E94240B8091E2008460809388
:10586000E2008091E10080FF1BC08091E20080FF98
:1058700017C08091E2008E7F8093E2008091E20069
:1058800080618093E2008091D80080628093D8008C
:1058900019BC85E080934E038AE092E10E94B7092B
:1058A0008091E10084FF2FC08091E20084FF2BC033
:1058B00080E189BD82E189BD89B5982F917080FF13
:1058C000FBCF8091D8008F7D8093D8008091E1003C
:1058D0008F7E8093E1008091E2008F7E8093E200D2
:1058E0008091E20081608093E20080914F038823E1
:1058F00009F489C084E080934E038EE092E10E9417
:10590000B70980914E038091E10083FF2BC0809105
:10591000E20083FF27C08091E100877F8093E10050
:1059200082E080934E0310924F038091E1008E7FBE
:105930008093E1008091E2008E7F8093E20080916D
:10594000E20080618093E20042E060E080E00E943B
:10595000F20A8091F00088608093F00082E192E189
:105960000E94B709FF91EF91BF91AF919F918F91E5
:105970007F916F915F914F913F912F910F900FBE4B
:105980000F901F9018951092400380913F03882339
:1059900009F43BCF80914E038430C1F49091E9002B
:1059A0009F702091EC00822F817020FD80E8892B70
:1059B00095E09093E9009091EB0090FF04C09091E6
:1059C000EE0097FD08C08F708093E90010923F03AE
:1059D0001CCF1092F1009091E80095FDFACF9091C4
:1059E000E80090FFF0CF9091E8009E779093E80058
:1059F000EACF19BC10924E0386E092E10E94B709EB
:105A0000109241032ECF8091E30087FD93E09093A5
:105A10004E0373CF78941F921FB61F9211248F9359
:105A20009F93AF93BF938091370390913803A091D8
:105A30003903B0913A030196A11DB11D809337033C
:105A400090933803A0933903B0933A03BF91AF9179
:105A50009F918F911F901FBE1F9018951F921FB688
:105A60001F9211248F939F93AF93BF93809136031E
:105A7000811113C08091370390913803A0913903AD
:105A8000B0913A034196A11DB11D809337039093C5
:105A90003803A0933903B0933A03BF91AF919F911C
:105AA0008F911F901FBE1F901895CDB7DEB7E69758
:105AB0000FB6F894DEBF0FBECDBF85B7806885BF37
:105AC00085B7806885BF84B7877F84BF0FB6F89499
:105AD000A8958091600088618093600010926000BA
:105AE0000FBE80E890E00FB6F89480936100909329
:105AF00061000FBE83ED90E190930902809308024C
:105B00000E94590A0E94240B8091E20084608093D5
:105B1000E200789480914E038823A1F01091E9006F
:105B20001F709091EC00892F817090FD80E8182BF8
:105B30001092E9008091E80083FD0E94A31C1F7071
:105B40001093E90082E084BD93E095BD9AEF97BD84
:105B500080936E000E945515811102C00E94AC1402
:105B600003EB11E048EBE42E41E0F42ED8018D91D7
:105B70008D018F3F11F00E942B0EE016F106B1F758
:105B800008EB11E039ECE32E31E0F32EF8018191BE
:105B90008F018F3F11F00E942B0EE016F106B1F736
:105BA00084E1E8EAF2E0DF01282F1D922A95E9F767
:105BB000ECE7F2E0DF011D928A95E9F70E948B2B5A
:105BC000811102C00E942C1C82E090E00E943635B8
:105BD00080932A030E946E15909391028093900205
:105BE0000E94FB19EFE3FCE93197F1F700C00000D8
:105BF0000E94FB198091A80280FF08C06FEF7FEF21
:105C000090E080E00E9468350E94B71183E090E048
:105C10000E9436350E94BD1B209A289880919202DE
:105C20008111DDC080912A0380FF14C08BE994E0CC
:105C30009F938F930E94500A80912A030F900F9098
:105C400080FF08C085E894E09F938F930E94500ADC
:105C50000F900F900E948B2B811110C080912A030E
:105C600080FF08C08DE594E09F938F930E94500AB7
:105C70000F900F900E942C1C0E94EB1988E090E07E
:105C80000E943E356093240370932503809326037E
:105C9000909327036E7FD1F480912A0380FF08C080
:105CA00084E194E09F938F930E94500A0F900F908D
:105CB0000E94EB1988E090E00E943E356093240337
:105CC0007093250380932603909327030E943C0C36
:105CD00080912A0380FF76C08BEF93E09F938F9390
:105CE0000E94500A80912A030F900F9080FF6AC093
:105CF0008091240381701F928F938EED93E09F9388
:105D00008F930E94500A80912A030F900F900F905A
:105D10000F9080FF57C08091240386951F928F9328
:105D200083EC93E09F938F930E94500A80912A0303
:105D30000F900F900F900F9080FF44C0809125032B
:105D40001F928F9389EA93E09F938F930E94500A4A
:105D500080912A030F900F900F900F9080FF32C018
:105D6000809126031F928F938FE893E09F938F93E8
:105D70000E94500A80912A030F900F900F900F906D
:105D800080FF20C0809127031F928F9385E793E0C7
:105D90009F938F930E94500A80912A030F900F9037
:105DA0000F900F9080FF0EC0809128031F928F9359
:105DB00089E593E09F938F930E94500A0F900F9074
:105DC0000F900F901092D0028091240380FF04C0A6
:105DD00060E086950E94581981E08093920284E0E9
:105DE00091E0909333038093320380914E0385308A
:105DF00089F482EB94E00E94B70900E112E18091FE
:105E00004E03853009F44EC00E94971C0E94280C56
:105E10000E94B5100E94FB19882359F08FB7F8949F
:105E200040913703509138036091390370913A03E0
:105E30008FBFA8EAB2E0BCA7ABA7E3E9F2E0FEA7F8
:105E4000EDA7B8ABAFA710E000E00EABAFA5B8A9C7
:105E50008D909D90AD90BD90B8ABAFA7EDA5FEA580
:105E60004190519061907190FEA7EDA7481459049C
:105E70006A047B0409F059C00F5F1F4F05301105FC
:105E800021F78FEF8EA38FA318A60E94F00B8160DD
:105E9000782F9AA789A74EA15FA168A58AA50E941D
:105EA000062B88C080914E03843039F180E00E9437
:105EB000B5101092360388E190E0A0E40FB6F89494
:105EC000A895809360000FBEA093600083B7817F88
:105ED000846083BF83B7816083BF7894889583B7DC
:105EE0008E7F83BF0FB6F894A8958091600088617B
:105EF00080936000109260000FBE80914D03882354
:105F000009F47DCF0E94FB19E8EAF2E081919191BA
:105F1000A191B191892B8A2B8B2B09F078C48CEB42
:105F200092E08E179F0791F76ACF80912A0381FD37
:105F30006EC1482459246A247B2480E0C12CD12CD2
:105F40007601C394B301A2014C215D216E217F2112
:105F5000452B462B472B09F4B7C189A32EA92AA3A9
:105F60008C209D20AE20BF2081E089288A288B28A4
:105F700009F480E08BA30E94F00B8160782F9DA331
:105F80008CA349A15AA16BA18DA10E94062BF801F7
:105F9000EE0FFF1FEE0FFF1FED56FD4F8081918129
:105FA000A281B3818C259D25AE25BF258083918359
:105FB000A283B3838091D0028823D1F18091CF0254
:105FC000E0912403E695E81BE093CB02823009F0D0
:105FD00084C1F0E0E150FB4FE4910E2F10E0A1E10D
:105FE000EA2EA4E1FA2E8091CC02882361F010926F
:105FF000CC020E94F00B9093CA028093C9021092C7
:10600000CE021092CD020E94F00BE091C902F091F5
:10601000CA028E1B9F0B8F3F9F4750F4E00FF11F6A
:10602000F093CA02E093C90289EC92E0F701099566
:1060300086E0E3ECF2E0DE01119601900D928A9584
:10604000E1F71092C5021092C6021092C702109298
:10605000C8028B819C81892B91F08091C102909123
:10606000C2020E94E10BAC019091BE02992309F497
:10607000A0C1809122018417150608F4A8C18D8162
:106080009E81892B09F44AC08091BF029091C00281
:106090000E94E10B9C019091BC02992309F4D6C3A4
:1060A00021353105D8F19F3F19F09F5F9093BC02D5
:1060B0001D81112359F00E945A0D9FEF11160CF407
:1060C00091E0899F802D11248093C7021E811123A6
:1060D00059F00E945A0D9FEF11160CF491E0899F20
:1060E000802D11248093C8023091C7023323B1F070
:1060F0002091C802222391F045EB3403C001112402
:10610000992309F4A5C19093C70245EB240390019C
:106110001124332309F4A0C13093C80246E050E0B3
:10612000BE016F5F7F4F83EC92E00E942935892B7F
:1061300061F48091C5029091C602892B9091C702AB
:10614000892B9091C802892B11F00E94CE1686E00F
:10615000FE013196A3ECB2E001900D928A95E1F731
:106160000E94280C182F8091A702181739F110935C
:10617000A70280912A0382FF1EC080FF1CC08AE014
:1061800095E00E94B70980912A0380FF14C01F92F6
:106190001F9385E095E09F938F930E94500A809112
:1061A0002A030F900F900F900F9080FF04C083E0A0
:1061B00095E00E94B709812F0E94B51080914E038F
:1061C000843009F012CE83E08093E9008091E800EA
:1061D00082FF0BCE8091E80090E085FF06C00E9410
:1061E000780A882309F43CC191E08091E8008B771C
:1061F0008093E800992309F4F8CDE981E150E33177
:1062000008F0B1C1F0E0E750FA4C0C946D3487EC23
:1062100094E00E94B70988EA92E09AAB89AB312CEE
:10622000212C3F922F92A2ECB4E0BF93AF930E9437
:10623000500A8FEB94E00E94B709A9A9BAA9CD90A2
:10624000DD90ED90FD90BAABA9AB8C2D0E94BB10F8
:106250008CAB8D2D0E94BB108DAB6701EE24FF240B
:106260008C2D0E94BB108BAB8D2D0E94BB10BCA946
:10627000EDA95B2F4E2F70E060E0BA01552744274F
:10628000FBA99F2FB0E0A0E0842B952BA62BB72B6A
:10629000BF93AF939F938F9388EB94E09F938F93DB
:1062A0000E94500A86EB94E00E94B709BFEF2B1AB8
:1062B0003B0A0FB6F894DEBF0FBECDBFF5E02F1638
:1062C000310409F0AECF35CE8F5FCC0CDD1CEE1C57
:1062D000FF1C813109F036CECFCD863059F4F0E085
:1062E000E450FB4FE4910E2F10E0F1E0EF2EF4E1CB
:1062F000FF2E79CE893061F4E695F0E0E750FB4F50
:10630000E4910E2F10E0E5E7EE2EE3E1FE2E6BCEDA
:106310008F3061F4E695F0E0EA50FB4FE4910E2FE8
:1063200010E070E1E72E73E1F72E5DCE853159F470
:10633000F0E0ED50FB4FE4910E2F10E062ECE62E02
:1063400062E1F62E50CE08E210E037E4E32E32E1AF
:10635000F32E883109F447CE833249F4E1EFF4E0BB
:106360000591149150EBE52E53E1F52E3CCE04EF50
:1063700011E020E1E22E22E1F22E843209F433CE44
:1063800000ED17E09BE3E92E9CE0F92E853209F041
:106390002ACE8E2F63E00E942B34E92FF0E0E251E9
:1063A000FB4FE4910E2F10E047E7E42E47E1F42E77
:1063B0001ACE20912301FAE02F9F90011124241777
:1063C000350708F05CCE9F5F9093BE0202C09F3FEE
:1063D000D1F71B81112359F00E94930D9FEF1116E5
:1063E0000CF491E0899F802D11248093C5021C81BB
:1063F000112359F00E94930D9FEF11160CF491E0B8
:10640000899F802D11248093C6023091C5023323C9
:1064100009F435CE2091C602222309F430CE45EB93
:106420003403C0011124992359F09093C50245EB20
:10643000240390011124332339F03093C6021FCE78
:1064400081E08093C502F3CF81E08093C60217CE2E
:1064500081E08093C70259CE81E08093C8025ECE6E
:1064600080E2E82EF12C8E010F5F1F4F8091E80033
:1064700085FD0AC08091E8008B778093E8000E9438
:10648000780A882399F3B0CE8091F100D8018D93DA
:106490008D01B1E0EB1AF10849F7A6CE1A8289E026
:1064A0008B831AC08A81823009F4C7C18330D9F145
:1064B000813009F058C02FB7F8946091370370917C
:1064C00038038091390390913A032FBF0E947334AF
:1064D0006B837C838D839E8380914E03843009F08F
:1064E00084CC1091E9001F709091EC00892F81708D
:1064F00090FD80E8182B82E08093E9008091E8000D
:1065000080FF0DC050E040E060E270E0CE010196F7
:106510000E94A90A8091E8008E778093E8001F709E
:106520001093E90062CCFE013196ABA5BCA54D915C
:106530005D916D917D91BCA7ABA76283538344832A
:106540003396AC5BB24089F7C7CF8A81823059F469
:106550006B817C818D819E810E94733486E290E004
:106560000E944A35B9CF8FEF8983B6CF4C816B81BA
:106570008A810E94BC149827892798279E838D833F
:10658000ABCF2D813E813227232732274C816B816F
:106590008A810E943514A0CF0E945B149DCF8A810E
:1065A0008138C9F060F4803809F096CF20E04B8143
:1065B00060912603809125030E9424188DCF823894
:1065C00009F44CC0833809F087CF20E040912703BD
:1065D0006C818B81F1CF60E08B810E9458192B81F7
:1065E00090912A038091240321111FC08E7F8093F4
:1065F000240390FF0CC01F921F9285E195E09F93AA
:106600008F930E94500A0F900F900F900F900E944E
:10661000BF164FEF80E792E0415080409040E1F795
:1066200000C000000E94DB1157CF816080932403DB
:1066300090FF0DC01F9281E08F938FE495E09F93B0
:106640008F930E94500A0F900F900F900F9080919F
:10665000240360E086950E9458193ECF8B81809379
:10666000280390912A0390FF37CF1F928F9388E8D9
:1066700095E09F938F930E94500A0F900F900F9078
:106680000F902ACF8A81813899F030F4803809F050
:1066900023CF8091270304CF823891F0833809F00B
:1066A0001BCF809125038B83809126038C8314CF8D
:1066B0008091240380FF02C08695F2CE80E0F0CE68
:1066C00080912803EDCE6091240370912503809181
:1066D0002603909127030E941118FECE80E18A8341
:1066E000FBCE81E08A8381E3DBCE0A811B81102708
:1066F00001271027DE0111966D01EC80FD01EE0DE2
:10670000F11D7F01C80181539D4FCE14DF0409F4B0
:10671000E3CE0133F1E01F0758F40E943635D6016D
:1067200014968C930F5F1F4FFFEFCF1ADF0AEACF4B
:10673000F6011482F7CF0A811B8110270127102749
:10674000CE0101966C01EC80E00EF12EF11CC80127
:1067500081539D4FE016F10609F4BECE0133A1E04E
:106760001A0720F4F60164810E944A35FFEFCF1A20
:10677000DF0A0F5F1F4FEBCF0E942514ADCE84E0E0
:10678000AECF0A811B81102701271027CE01019669
:106790006C01EC80DC01AE0DB11D7D01C801879656
:1067A000EC14FD0409F498CE083AB2E01B0750F44B
:1067B0000E943635F60184830F5F1F4FBFEFCB1A5F
:1067C000DB0AECCFD60114961C92F6CF0A811B810E
:1067D000102701271027FE0131966F01EC80E00E93
:1067E000F12EF11CC8018796E016F10609F474CE6B
:1067F000083AF2E01F0728F4D60114966C910E9423
:106800004A35BFEFCB1ADB0A0F5F1F4FEBCF09BD35
:1068100019BD09B400FEFDCF8091D8008F7D809313
:10682000D8008091E00082608093E0008091E000D9
:1068300081FDFCCF0E94971CE2CA86E290E00E9494
:1068400036351B821C821D828E8346CE2B3031054D
:1068500008F02BCC63CC991B79E004C0991F9617E4
:1068600008F0961B881F7A95C9F78095089587FBD5
:10687000082E062687FD819567FD61950E942B34C1
:106880000EF4919507FC81950895AA1BBB1B51E15D
:1068900007C0AA1FBB1FA617B70710F0A61BB70B90
:1068A000881F991F5A95A9F780959095BC01CD0135
:1068B000089597FB072E16F4009407D077FD09D0B2
:1068C0000E94453407FC05D03EF4909581959F4F7A
:1068D0000895709561957F4F0895EE0FFF1F059005
:1068E000F491E02D0994692796276927782787274F
:1068F000782708950E94D235332312F48A1B9B0B0C
:106900000C9484340E94D235B7FF0895821B930BF8
:1069100008952F923F924F925F926F927F928F9243
:106920009F92AF92BF92CF92DF92EF92FF920F931E
:106930001F93CF93DF93CDB7DEB7CA1BDB0B0FB628
:10694000F894DEBF0FBECDBF09942A8839884888E5
:106950005F846E847D848C849B84AA84B984C8847B
:10696000DF80EE80FD800C811B81AA81B981CE0F72
:10697000D11D0FB6F894DEBF0FBECDBFED01089557
:106980008F929F92AF92BF92CF92DF92EF92FF923F
:10699000CF93DF93EC01688179818A819B816115B6
:1069A00071058105910521F464E279ED8BE597E0AD
:1069B0002DE133EF41E050E00E947E3549015A015C
:1069C0009B01AC01A7EAB1E40E949D356B017C01FB
:1069D000ACEEB4EFA50194010E94AB35DC01CB0114
:1069E0008C0D9D1DAE1DBF1DB7FF03C00197A109F2
:1069F000B04888839983AA83BB839F77DF91CF9127
:106A0000FF90EF90DF90CF90BF90AF909F908F90CE
:106A100008950E94C034089580E091E00E94C0343F
:106A20000895B0E0A0E08093000190930101A0934D
:106A30000201B09303010895FC014150504030F031
:106A400001900616D1F73197CF010895882799272D
:106A50000895FB01DC0104C08D910190801921F49F
:106A600041505040C8F7881B990B0895F999FECF03
:106A700092BD81BDF89A992780B50895A6E1B0E04E
:106A800044E050E00C947035A8E1B0E042E050E002
:106A90000C947035262FF999FECF92BD81BDF89ADE
:106AA000019700B4021639F01FBA20BD0FB6F89452
:106AB000FA9AF99A0FBE08950396272F0E944B3534
:106AC0000E944A35252F0E944B35242F0C944B35BC
:106AD0000196272F0E944B350C944A35DC01CB01DF
:106AE000FC01F999FECF06C0F2BDE1BDF89A3196DE
:106AF00000B40D9241505040B8F70895052E97FB11
:106B00001EF400940E94953557FD07D00E94B035C1
:106B100007FC03D04EF40C94953550954095309574
:106B200021953F4F4F4F5F4F0895909580957095F9
:106B300061957F4F8F4F9F4F08950E94D235A59F3B
:106B4000900DB49F900DA49F800D911D1124089568
:106B5000B7FF0C949D350E949D35821B930B0895C1
:106B6000A1E21A2EAA1BBB1BFD010DC0AA1FBB1F51
:106B7000EE1FFF1FA217B307E407F50720F0A21BC3
:106B8000B30BE40BF50B661F771F881F991F1A9430
:106B900069F760957095809590959B01AC01BD015A
:106BA000CF010895A29FB001B39FC001A39F700DB4
:106BB000811D1124911DB29F700D811D1124911D05
:106BC0000895F894FFCF841DAC1D551FAC1D551FB3
:106BD000DF1D001E551FFE1E0B1FF425F4252F265A
:106BE0002F26C826E2265E265E26ED265A276B272C
:106BF0006B274E325232A532B632C132CC32CF324E
:106C000042336333B332B3326E33713375339B33F4
:086C1000BC33BF33C133E6338E
:106C180001000000DE0B8A11691164115F11DD0BA0
:106C280001191A1B1C1D1E1F202122010201280800
:106C38001E0A1401013F3F3F006D6B5F64656C6184
:106C480079006D6B5F696E74657276616C006D6B4F
:106C58005F6D61785F7370656564006D6B5F746903
:106C68006D655F746F5F6D6178006D6B5F776865E8
:106C7800656C5F6D61785F7370656564006D6B5FEF
:106C8800776865656C5F74696D655F746F5F6D616A
:106C98007800818283E200E900EA00B500B600B717
:106CA80000CD008301CC008A0192019401210223C6
:106CB8000224022502260227022A02B300B4006F2A
:106CC8000070003332F4F5F6F0F1F73190919293B9
:106CD80095949697343536666700010202020206DB
:106CE80006060909090909090F0F0F0F0F0F1515D6
:106CF80015181919191919191919191923242525D4
:106D08002525252540227B226B014901CE00AC00B8
:086D18002812411261127A12E7
:00000001FF
